 jaccesswalker

 Timestamp is 5fa5faeb (reproducible build file hash)

 Preferred load address is 0000000140000000

 Start         Length     Name                   Class
 0001:00000000 00008a00H .text$mn                CODE
 0001:00008a00 00000040H .text$mn$00             CODE
 0001:00008a40 00000053H .text$x                 CODE
 0002:00000000 000003a0H .idata$5                DATA
 0002:000003a0 00000038H .00cfg                  DATA
 0002:000003d8 00000008H .CRT$XCA                DATA
 0002:000003e0 00000008H .CRT$XCAA               DATA
 0002:000003e8 00000008H .CRT$XCZ                DATA
 0002:000003f0 00000008H .CRT$XIA                DATA
 0002:000003f8 00000008H .CRT$XIAA               DATA
 0002:00000400 00000008H .CRT$XIAC               DATA
 0002:00000408 00000008H .CRT$XIZ                DATA
 0002:00000410 00000008H .CRT$XPA                DATA
 0002:00000418 00000008H .CRT$XPZ                DATA
 0002:00000420 00000008H .CRT$XTA                DATA
 0002:00000428 00000008H .CRT$XTZ                DATA
 0002:00000430 00000000H .gehcont$y              DATA
 0002:00000430 00000000H .gfids$y                DATA
 0002:00000430 00001d50H .rdata                  DATA
 0002:00002180 00000000H .rdata$CastGuardVftablesA DATA
 0002:00002180 00000000H .rdata$CastGuardVftablesC DATA
 0002:00002180 000001f4H .rdata$r                DATA
 0002:00002374 000000b8H .rdata$voltmd           DATA
 0002:0000242c 0000033cH .rdata$zzzdbg           DATA
 0002:00002768 00000008H .rtc$IAA                DATA
 0002:00002770 00000008H .rtc$IZZ                DATA
 0002:00002778 00000008H .rtc$TAA                DATA
 0002:00002780 00000008H .rtc$TZZ                DATA
 0002:00002788 000005c8H .xdata                  DATA
 0002:00002d50 000000ecH .xdata$x                DATA
 0002:00002e3c 00000000H .edata                  DATA
 0002:00002e3c 00000118H .idata$2                DATA
 0002:00002f54 00000014H .idata$3                DATA
 0002:00002f68 000003a0H .idata$4                DATA
 0002:00003308 00000882H .idata$6                DATA
 0003:00000000 00000c48H .data                   DATA
 0003:00000c48 00000080H .data$r                 DATA
 0003:00000cc8 00000038H .data$rs                DATA
 0003:00000d00 00000ae0H .bss                    DATA
 0004:00000000 00000888H .pdata                  DATA
 0005:00000000 000001d0H .rsrc$01                DATA
 0005:000001d0 00000540H .rsrc$02                DATA

  Address         Publics by Value              Rva+Base               Lib:Object

 0000:00000000       __AbsoluteZero             0000000000000000     <absolute>
 0000:00000000       ___safe_se_handler_count   0000000000000000     <absolute>
 0000:00000000       ___safe_se_handler_table   0000000000000000     <absolute>
 0000:00000000       __arm64x_extra_rfe_table   0000000000000000     <absolute>
 0000:00000000       __arm64x_extra_rfe_table_size 0000000000000000     <absolute>
 0000:00000000       __arm64x_native_entrypoint 0000000000000000     <absolute>
 0000:00000000       __arm64x_redirection_metadata 0000000000000000     <absolute>
 0000:00000000       __arm64x_redirection_metadata_count 0000000000000000     <absolute>
 0000:00000000       __dynamic_value_reloc_table 0000000000000000     <absolute>
 0000:00000000       __enclave_config           0000000000000000     <absolute>
 0000:00000000       __guard_check_icall_a64n_fptr 0000000000000000     <absolute>
 0000:00000000       __guard_eh_cont_count      0000000000000000     <absolute>
 0000:00000000       __guard_eh_cont_table      0000000000000000     <absolute>
 0000:00000000       __guard_fids_count         0000000000000000     <absolute>
 0000:00000000       __guard_fids_table         0000000000000000     <absolute>
 0000:00000000       __guard_iat_count          0000000000000000     <absolute>
 0000:00000000       __guard_iat_table          0000000000000000     <absolute>
 0000:00000000       __guard_longjmp_count      0000000000000000     <absolute>
 0000:00000000       __guard_longjmp_table      0000000000000000     <absolute>
 0000:00000000       __hybrid_auxiliary_delayload_iat 0000000000000000     <absolute>
 0000:00000000       __hybrid_auxiliary_delayload_iat_copy 0000000000000000     <absolute>
 0000:00000000       __hybrid_auxiliary_iat     0000000000000000     <absolute>
 0000:00000000       __hybrid_auxiliary_iat_copy 0000000000000000     <absolute>
 0000:00000000       __hybrid_code_map          0000000000000000     <absolute>
 0000:00000000       __hybrid_code_map_count    0000000000000000     <absolute>
 0000:00000000       __hybrid_image_info_bitfield 0000000000000000     <absolute>
 0000:00000000       __x64_code_ranges_to_entry_points 0000000000000000     <absolute>
 0000:00000000       __x64_code_ranges_to_entry_points_count 0000000000000000     <absolute>
 0000:00000100       __guard_flags              0000000000000100     <absolute>
 0000:00000000       __ImageBase                0000000140000000     <linker-defined>
 0001:00000000       initializeAccessBridge     0000000140001000 f   AccessBridgeCalls.obj
 0001:000010d0       shutdownAccessBridge       00000001400020d0 f   AccessBridgeCalls.obj
 0001:00001120       IsJavaWindow               0000000140002120 f   AccessBridgeCalls.obj
 0001:00001160       GetAccessibleContextFromHWND 0000000140002160 f   AccessBridgeCalls.obj
 0001:000011a0       getHWNDFromAccessibleContext 00000001400021a0 f   AccessBridgeCalls.obj
 0001:000011e0       SetJavaShutdown            00000001400021e0 f   AccessBridgeCalls.obj
 0001:00001210       SetFocusGained             0000000140002210 f   AccessBridgeCalls.obj
 0001:00001240       SetFocusLost               0000000140002240 f   AccessBridgeCalls.obj
 0001:00001270       SetCaretUpdate             0000000140002270 f   AccessBridgeCalls.obj
 0001:000012a0       SetMouseClicked            00000001400022a0 f   AccessBridgeCalls.obj
 0001:000012d0       SetMouseEntered            00000001400022d0 f   AccessBridgeCalls.obj
 0001:00001300       SetMouseExited             0000000140002300 f   AccessBridgeCalls.obj
 0001:00001330       SetMousePressed            0000000140002330 f   AccessBridgeCalls.obj
 0001:00001360       SetMouseReleased           0000000140002360 f   AccessBridgeCalls.obj
 0001:00001390       SetMenuCanceled            0000000140002390 f   AccessBridgeCalls.obj
 0001:000013c0       SetMenuDeselected          00000001400023c0 f   AccessBridgeCalls.obj
 0001:000013f0       SetMenuSelected            00000001400023f0 f   AccessBridgeCalls.obj
 0001:00001420       SetPopupMenuCanceled       0000000140002420 f   AccessBridgeCalls.obj
 0001:00001450       SetPopupMenuWillBecomeInvisible 0000000140002450 f   AccessBridgeCalls.obj
 0001:00001480       SetPopupMenuWillBecomeVisible 0000000140002480 f   AccessBridgeCalls.obj
 0001:000014b0       SetPropertyNameChange      00000001400024b0 f   AccessBridgeCalls.obj
 0001:000014e0       SetPropertyDescriptionChange 00000001400024e0 f   AccessBridgeCalls.obj
 0001:00001510       SetPropertyStateChange     0000000140002510 f   AccessBridgeCalls.obj
 0001:00001540       SetPropertyValueChange     0000000140002540 f   AccessBridgeCalls.obj
 0001:00001570       SetPropertySelectionChange 0000000140002570 f   AccessBridgeCalls.obj
 0001:000015a0       SetPropertyTextChange      00000001400025a0 f   AccessBridgeCalls.obj
 0001:000015d0       SetPropertyCaretChange     00000001400025d0 f   AccessBridgeCalls.obj
 0001:00001600       SetPropertyVisibleDataChange 0000000140002600 f   AccessBridgeCalls.obj
 0001:00001630       SetPropertyChildChange     0000000140002630 f   AccessBridgeCalls.obj
 0001:00001660       SetPropertyActiveDescendentChange 0000000140002660 f   AccessBridgeCalls.obj
 0001:00001690       SetPropertyTableModelChange 0000000140002690 f   AccessBridgeCalls.obj
 0001:000016c0       ReleaseJavaObject          00000001400026c0 f   AccessBridgeCalls.obj
 0001:00001700       GetVersionInfo             0000000140002700 f   AccessBridgeCalls.obj
 0001:00001740       GetAccessibleContextAt     0000000140002740 f   AccessBridgeCalls.obj
 0001:000017a0       GetAccessibleContextWithFocus 00000001400027a0 f   AccessBridgeCalls.obj
 0001:000017e0       GetAccessibleContextInfo   00000001400027e0 f   AccessBridgeCalls.obj
 0001:00001820       GetAccessibleChildFromContext 0000000140002820 f   AccessBridgeCalls.obj
 0001:00001860       GetAccessibleParentFromContext 0000000140002860 f   AccessBridgeCalls.obj
 0001:000018a0       GetAccessibleTextInfo      00000001400028a0 f   AccessBridgeCalls.obj
 0001:000018f0       GetAccessibleTextItems     00000001400028f0 f   AccessBridgeCalls.obj
 0001:00001940       GetAccessibleTextSelectionInfo 0000000140002940 f   AccessBridgeCalls.obj
 0001:00001980       GetAccessibleTextAttributes 0000000140002980 f   AccessBridgeCalls.obj
 0001:000019d0       GetAccessibleTextRect      00000001400029d0 f   AccessBridgeCalls.obj
 0001:00001a20       GetAccessibleTextLineBounds 0000000140002a20 f   AccessBridgeCalls.obj
 0001:00001a80       GetAccessibleTextRange     0000000140002a80 f   AccessBridgeCalls.obj
 0001:00001ae0       getAccessibleTableInfo     0000000140002ae0 f   AccessBridgeCalls.obj
 0001:00001b20       getAccessibleTableCellInfo 0000000140002b20 f   AccessBridgeCalls.obj
 0001:00001b80       getAccessibleTableRowHeader 0000000140002b80 f   AccessBridgeCalls.obj
 0001:00001bc0       getAccessibleTableColumnHeader 0000000140002bc0 f   AccessBridgeCalls.obj
 0001:00001c00       getAccessibleTableRowDescription 0000000140002c00 f   AccessBridgeCalls.obj
 0001:00001c40       getAccessibleTableColumnDescription 0000000140002c40 f   AccessBridgeCalls.obj
 0001:00001c80       getAccessibleTableRowSelectionCount 0000000140002c80 f   AccessBridgeCalls.obj
 0001:00001cc0       isAccessibleTableRowSelected 0000000140002cc0 f   AccessBridgeCalls.obj
 0001:00001d00       getAccessibleTableRowSelections 0000000140002d00 f   AccessBridgeCalls.obj
 0001:00001d50       getAccessibleTableColumnSelectionCount 0000000140002d50 f   AccessBridgeCalls.obj
 0001:00001d90       isAccessibleTableColumnSelected 0000000140002d90 f   AccessBridgeCalls.obj
 0001:00001dd0       getAccessibleTableColumnSelections 0000000140002dd0 f   AccessBridgeCalls.obj
 0001:00001e20       getAccessibleTableRow      0000000140002e20 f   AccessBridgeCalls.obj
 0001:00001e70       getAccessibleTableColumn   0000000140002e70 f   AccessBridgeCalls.obj
 0001:00001ec0       getAccessibleTableIndex    0000000140002ec0 f   AccessBridgeCalls.obj
 0001:00001f10       getAccessibleRelationSet   0000000140002f10 f   AccessBridgeCalls.obj
 0001:00001f50       getAccessibleHypertext     0000000140002f50 f   AccessBridgeCalls.obj
 0001:00001f90       activateAccessibleHyperlink 0000000140002f90 f   AccessBridgeCalls.obj
 0001:00001fd0       getAccessibleHyperlinkCount 0000000140002fd0 f   AccessBridgeCalls.obj
 0001:00002010       getAccessibleHypertextExt  0000000140003010 f   AccessBridgeCalls.obj
 0001:00002060       getAccessibleHypertextLinkIndex 0000000140003060 f   AccessBridgeCalls.obj
 0001:000020b0       getAccessibleHyperlink     00000001400030b0 f   AccessBridgeCalls.obj
 0001:00002100       getAccessibleKeyBindings   0000000140003100 f   AccessBridgeCalls.obj
 0001:00002140       getAccessibleIcons         0000000140003140 f   AccessBridgeCalls.obj
 0001:00002180       getAccessibleActions       0000000140003180 f   AccessBridgeCalls.obj
 0001:000021c0       doAccessibleActions        00000001400031c0 f   AccessBridgeCalls.obj
 0001:00002210       IsSameObject               0000000140003210 f   AccessBridgeCalls.obj
 0001:00002250       setTextContents            0000000140003250 f   AccessBridgeCalls.obj
 0001:00002290       getParentWithRole          0000000140003290 f   AccessBridgeCalls.obj
 0001:000022d0       getParentWithRoleElseRoot  00000001400032d0 f   AccessBridgeCalls.obj
 0001:00002310       getTopLevelObject          0000000140003310 f   AccessBridgeCalls.obj
 0001:00002350       getObjectDepth             0000000140003350 f   AccessBridgeCalls.obj
 0001:00002390       getActiveDescendent        0000000140003390 f   AccessBridgeCalls.obj
 0001:000023d0       GetCurrentAccessibleValueFromContext 00000001400033d0 f   AccessBridgeCalls.obj
 0001:00002420       GetMaximumAccessibleValueFromContext 0000000140003420 f   AccessBridgeCalls.obj
 0001:00002470       GetMinimumAccessibleValueFromContext 0000000140003470 f   AccessBridgeCalls.obj
 0001:000024c0       GetAccessibleSelectionFromContext 00000001400034c0 f   AccessBridgeCalls.obj
 0001:00002500       GetAccessibleSelectionCountFromContext 0000000140003500 f   AccessBridgeCalls.obj
 0001:00002540       IsAccessibleChildSelectedFromContext 0000000140003540 f   AccessBridgeCalls.obj
 0001:00002580       RemoveAccessibleSelectionFromContext 0000000140003580 f   AccessBridgeCalls.obj
 0001:000025c0       SelectAllAccessibleSelectionFromContext 00000001400035c0 f   AccessBridgeCalls.obj
 0001:00002600       getVirtualAccessibleName   0000000140003600 f   AccessBridgeCalls.obj
 0001:00002650       requestFocus               0000000140003650 f   AccessBridgeCalls.obj
 0001:00002690       selectTextRange            0000000140003690 f   AccessBridgeCalls.obj
 0001:000026e0       getTextAttributesInRange   00000001400036e0 f   AccessBridgeCalls.obj
 0001:00002740       getVisibleChildrenCount    0000000140003740 f   AccessBridgeCalls.obj
 0001:00002780       getVisibleChildren         0000000140003780 f   AccessBridgeCalls.obj
 0001:000027d0       setCaretPosition           00000001400037d0 f   AccessBridgeCalls.obj
 0001:00002810       getCaretLocation           0000000140003810 f   AccessBridgeCalls.obj
 0001:00002860       getEventsWaiting           0000000140003860 f   AccessBridgeCalls.obj
 0001:00002890       addAccessibleSelectionFromContext 0000000140003890 f   AccessBridgeCalls.obj
 0001:000028d0       clearAccessibleSelectionFromContext 00000001400038d0 f   AccessBridgeCalls.obj
 0001:00002900       printError                 0000000140003900 f   AccessBridgeDebug.obj
 0001:00002a60       PrintDebugString           0000000140003a60 f   AccessBridgeDebug.obj
 0001:00002af0       wPrintJavaDebugString      0000000140003af0 f   AccessBridgeDebug.obj
 0001:00002b80       wPrintDebugString          0000000140003b80 f   AccessBridgeDebug.obj
 0001:00002c10       initializeFileLogger       0000000140003c10 f   AccessBridgeDebug.obj
 0001:00002d90       finalizeFileLogger         0000000140003d90 f   AccessBridgeDebug.obj
 0001:00002dd0       getTimeStamp               0000000140003dd0 f   AccessBridgeDebug.obj
 0001:00002e20       PrintJavaDebugString2      0000000140003e20 f   AccessBridgeDebug.obj
 0001:00002ea0       __local_stdio_printf_options 0000000140003ea0 f i AccessBridgeDebug.obj
 0001:00002eb0       _vfprintf_l                0000000140003eb0 f i AccessBridgeDebug.obj
 0001:00002f00       _vfwprintf_l               0000000140003f00 f i AccessBridgeDebug.obj
 0001:00002f50       fprintf                    0000000140003f50 f i AccessBridgeDebug.obj
 0001:00002fa0       printf                     0000000140003fa0 f i AccessBridgeDebug.obj
 0001:00003000       vfprintf                   0000000140004000 f i AccessBridgeDebug.obj
 0001:00003030       vfwprintf                  0000000140004030 f i AccessBridgeDebug.obj
 0001:00003060       ?initBroadcastMessageIDs@@YAHXZ 0000000140004060 f   AccessBridgeMessages.obj
 0001:000030b0       ?getTimeAndDate@@YAPEADXZ  00000001400040b0 f   AccessInfo.obj
 0001:00003180       ?displayAndLog@@YAXPEAUHWND__@@HPEAU_iobuf@@PEADZZ 0000000140004180 f   AccessInfo.obj
 0001:000032a0       ?logString@@YAXPEAU_iobuf@@PEBDZZ 00000001400042a0 f   AccessInfo.obj
 0001:00003370       ?getAccessibleInfo@@YAPEADJ_JPEADH@Z 0000000140004370 f   AccessInfo.obj
 0001:000033c0       ?getAccessibleInfo@@YAPEADJ_JHHPEADH@Z 00000001400043c0 f   AccessInfo.obj
 0001:00005df0       ?appendToBuffer@@YAHPEAD_KPEBDZZ 0000000140006df0 f   AccessInfo.obj
 0001:00005f00       snprintf                   0000000140006f00 f i AccessInfo.obj
 0001:00005f60       vsnprintf                  0000000140006f60 f i AccessInfo.obj
 0001:00005fe0       WinMain                    0000000140006fe0 f   jaccesswalker.obj
 0001:000060a0       ??0AccessibleNode@@QEAA@J_JPEAV0@PEAUHWND__@@PEAU_TREEITEM@@@Z 00000001400070a0 f   jaccesswalker.obj
 0001:00006110       ??1AccessibleNode@@QEAA@XZ 0000000140007110 f   jaccesswalker.obj
 0001:00006140       ?setAccessibleName@AccessibleNode@@QEAAXPEAD@Z 0000000140007140 f   jaccesswalker.obj
 0001:00006180       ?setAccessibleRole@AccessibleNode@@QEAAXPEAD@Z 0000000140007180 f   jaccesswalker.obj
 0001:000061c0       ?displayAPIWindow@AccessibleNode@@QEAAHXZ 00000001400071c0 f   jaccesswalker.obj
 0001:00006320       ??0Jaccesswalker@@QEAA@H@Z 0000000140007320 f   jaccesswalker.obj
 0001:000065d0       ?buildAccessibilityTree@Jaccesswalker@@QEAAXXZ 00000001400075d0 f   jaccesswalker.obj
 0001:00006610       ?addComponentNodes@Jaccesswalker@@QEAAXJ_JPEAVAccessibleNode@@PEAUHWND__@@PEAU_TREEITEM@@2@Z 0000000140007610 f   jaccesswalker.obj
 0001:00006960       ?WinProc@@YA_JPEAUHWND__@@I_K_J@Z 0000000140007960 f   jaccesswalker.obj
 0001:00006c70       ?EnumWndProc@@YAHPEAUHWND__@@_J@Z 0000000140007c70 f   jaccesswalker.obj
 0001:00006da0       ?EnumChildProc@@YAHPEAUHWND__@@_J@Z 0000000140007da0 f   jaccesswalker.obj
 0001:00006e60       ?CreateATreeView@@YAPEAUHWND__@@PEAU1@@Z 0000000140007e60 f   jaccesswalker.obj
 0001:00006f20       ?AccessInfoWindowProc@@YA_JPEAUHWND__@@IIJ@Z 0000000140007f20 f   jaccesswalker.obj
 0001:000070e0       ?IsInaccessibleJavaWindow@@YAHQEAUHWND__@@@Z 00000001400080e0 f   jaccesswalker.obj
 0001:0000776c       ??_U@YAPEAX_K@Z            000000014000876c f   MSVCRT:new_array.obj
 0001:00007774       ??3@YAXPEAX_K@Z            0000000140008774 f   MSVCRT:delete_scalar_size.obj
 0001:00007774       ??_V@YAXPEAX@Z             0000000140008774 f   MSVCRT:delete_array.obj
 0001:0000777c       __raise_securityfailure    000000014000877c f   MSVCRT:gs_report.obj
 0001:000077b0       __report_gsfailure         00000001400087b0 f   MSVCRT:gs_report.obj
 0001:00007884       __report_rangecheckfailure 0000000140008884 f   MSVCRT:gs_report.obj
 0001:00007898       __report_securityfailure   0000000140008898 f   MSVCRT:gs_report.obj
 0001:00007a1c       __GSHandlerCheck           0000000140008a1c f   MSVCRT:gshandler.obj
 0001:00007a3c       __GSHandlerCheckCommon     0000000140008a3c f   MSVCRT:gshandler.obj
 0001:00007ab0       __chkstk                   0000000140008ab0 f   MSVCRT:chkstk.obj
 0001:00007ab0       _alloca_probe              0000000140008ab0 f   MSVCRT:chkstk.obj
 0001:00007b10       __security_check_cookie    0000000140008b10 f   MSVCRT:amdsecgs.obj
 0001:00007b30       ??2@YAPEAX_K@Z             0000000140008b30 f   MSVCRT:new_scalar.obj
 0001:00007b6c       __GSHandlerCheck_EH4       0000000140008b6c f   MSVCRT:gshandlereh4.obj
 0001:00007e44       WinMainCRTStartup          0000000140008e44 f   MSVCRT:exe_winmain.obj
 0001:00007e58       ??3@YAXPEAX@Z              0000000140008e58 f   MSVCRT:delete_scalar.obj
 0001:00007e60       ??0bad_alloc@std@@QEAA@AEBV01@@Z 0000000140008e60 f i MSVCRT:throw_bad_alloc.obj
 0001:00007e9c       ??0bad_alloc@std@@QEAA@XZ  0000000140008e9c f i MSVCRT:throw_bad_alloc.obj
 0001:00007ebc       ??0bad_array_new_length@std@@QEAA@AEBV01@@Z 0000000140008ebc f i MSVCRT:throw_bad_alloc.obj
 0001:00007ef8       ??0bad_array_new_length@std@@QEAA@XZ 0000000140008ef8 f i MSVCRT:throw_bad_alloc.obj
 0001:00007f18       ??0exception@std@@QEAA@AEBV01@@Z 0000000140008f18 f i MSVCRT:throw_bad_alloc.obj
 0001:00007f4c       ??1bad_alloc@std@@UEAA@XZ  0000000140008f4c f i MSVCRT:throw_bad_alloc.obj
 0001:00007f4c       ??1bad_array_new_length@std@@UEAA@XZ 0000000140008f4c f i MSVCRT:throw_bad_alloc.obj
 0001:00007f60       ??_Ebad_alloc@std@@UEAAPEAXI@Z 0000000140008f60 f i MSVCRT:throw_bad_alloc.obj
 0001:00007f60       ??_Ebad_array_new_length@std@@UEAAPEAXI@Z 0000000140008f60 f i MSVCRT:throw_bad_alloc.obj
 0001:00007f60       ??_Eexception@std@@UEAAPEAXI@Z 0000000140008f60 f i MSVCRT:throw_bad_alloc.obj
 0001:00007f60       ??_Gbad_alloc@std@@UEAAPEAXI@Z 0000000140008f60 f i MSVCRT:throw_bad_alloc.obj
 0001:00007f60       ??_Gbad_array_new_length@std@@UEAAPEAXI@Z 0000000140008f60 f i MSVCRT:throw_bad_alloc.obj
 0001:00007f60       ??_Gexception@std@@UEAAPEAXI@Z 0000000140008f60 f i MSVCRT:throw_bad_alloc.obj
 0001:00007fa4       ?__scrt_throw_std_bad_alloc@@YAXXZ 0000000140008fa4 f   MSVCRT:throw_bad_alloc.obj
 0001:00007fc4       ?__scrt_throw_std_bad_array_new_length@@YAXXZ 0000000140008fc4 f   MSVCRT:throw_bad_alloc.obj
 0001:00007fe4       ?what@exception@std@@UEBAPEBDXZ 0000000140008fe4 f i MSVCRT:throw_bad_alloc.obj
 0001:00007ff8       __scrt_acquire_startup_lock 0000000140008ff8 f   MSVCRT:utility.obj
 0001:00008034       __scrt_initialize_crt      0000000140009034 f   MSVCRT:utility.obj
 0001:00008070       __scrt_initialize_onexit_tables 0000000140009070 f   MSVCRT:utility.obj
 0001:000080fc       __scrt_is_nonwritable_in_current_image 00000001400090fc f   MSVCRT:utility.obj
 0001:00008194       __scrt_release_startup_lock 0000000140009194 f   MSVCRT:utility.obj
 0001:000081b8       __scrt_uninitialize_crt    00000001400091b8 f   MSVCRT:utility.obj
 0001:000081e4       _onexit                    00000001400091e4 f   MSVCRT:utility.obj
 0001:00008220       atexit                     0000000140009220 f   MSVCRT:utility.obj
 0001:00008238       __security_init_cookie     0000000140009238 f   MSVCRT:gs_support.obj
 0001:000082e4       __scrt_exe_initialize_mta  00000001400092e4 f   MSVCRT:utility_desktop.obj
 0001:000082e4       __scrt_initialize_winrt    00000001400092e4 f   MSVCRT:utility_desktop.obj
 0001:000082e4       __scrt_stub_for_initialize_mta 00000001400092e4 f   MSVCRT:utility_desktop.obj
 0001:000082e4       _get_startup_commit_mode   00000001400092e4 f   MSVCRT:commit_mode.obj
 0001:000082e4       _get_startup_new_mode      00000001400092e4 f   MSVCRT:new_mode.obj
 0001:000082e4       _get_startup_thread_locale_mode 00000001400092e4 f   MSVCRT:thread_locale.obj
 0001:000082e4       _matherr                   00000001400092e4 f   MSVCRT:matherr.obj
 0001:000082e8       _get_startup_argv_mode     00000001400092e8 f   MSVCRT:argv_mode.obj
 0001:000082f0       _get_startup_file_mode     00000001400092f0 f   MSVCRT:file_mode.obj
 0001:000082f8       ?__scrt_initialize_type_info@@YAXXZ 00000001400092f8 f   MSVCRT:tncleanup.obj
 0001:00008308       __acrt_initialize          0000000140009308 f   MSVCRT:ucrt_stubs.obj
 0001:00008308       __acrt_uninitialize        0000000140009308 f   MSVCRT:ucrt_stubs.obj
 0001:00008308       __scrt_stub_for_acrt_initialize 0000000140009308 f   MSVCRT:ucrt_stubs.obj
 0001:00008308       __scrt_stub_for_acrt_uninitialize 0000000140009308 f   MSVCRT:ucrt_stubs.obj
 0001:00008308       __vcrt_initialize          0000000140009308 f   MSVCRT:ucrt_stubs.obj
 0001:00008308       __vcrt_uninitialize        0000000140009308 f   MSVCRT:ucrt_stubs.obj
 0001:00008308       _should_initialize_environment 0000000140009308 f   MSVCRT:env_mode.obj
 0001:0000830c       _guard_check_icall_nop     000000014000930c f   MSVCRT:guard_support.obj
 0001:0000830c       _initialize_denormal_control 000000014000930c f   MSVCRT:denormal_control.obj
 0001:0000830c       _initialize_invalid_parameter_handler 000000014000930c f   MSVCRT:invalid_parameter_handler.obj
 0001:00008310       __local_stdio_scanf_options 0000000140009310 f i MSVCRT:default_local_stdio_options.obj
 0001:00008318       __scrt_initialize_default_local_stdio_options 0000000140009318 f   MSVCRT:default_local_stdio_options.obj
 0001:00008334       __scrt_is_user_matherr_present 0000000140009334 f   MSVCRT:matherr_detection.obj
 0001:00008340       __scrt_get_dyn_tls_init_callback 0000000140009340 f   MSVCRT:dyn_tls_init.obj
 0001:00008348       __scrt_get_dyn_tls_dtor_callback 0000000140009348 f   MSVCRT:dyn_tls_dtor.obj
 0001:00008350       __crt_debugger_hook        0000000140009350 f   MSVCRT:utility_desktop.obj
 0001:00008358       __scrt_fastfail            0000000140009358 f   MSVCRT:utility_desktop.obj
 0001:000084a0       __scrt_get_show_window_mode 00000001400094a0 f   MSVCRT:utility_desktop.obj
 0001:000084dc       __scrt_initialize_mta      00000001400094dc f   MSVCRT:utility_desktop.obj
 0001:000084e4       __scrt_is_managed_app      00000001400094e4 f   MSVCRT:utility_desktop.obj
 0001:00008538       __scrt_set_unhandled_exception_filter 0000000140009538 f   MSVCRT:utility_desktop.obj
 0001:00008548       __scrt_unhandled_exception_filter 0000000140009548 f   MSVCRT:utility_desktop.obj
 0001:000085a4       _RTC_Initialize            00000001400095a4 f   MSVCRT:initsect.obj
 0001:000085e0       _RTC_Terminate             00000001400095e0 f   MSVCRT:initsect.obj
 0001:0000861c       ??_Etype_info@@UEAAPEAXI@Z 000000014000961c f i MSVCRT:std_type_info_static.obj
 0001:0000861c       ??_Gtype_info@@UEAAPEAXI@Z 000000014000961c f i MSVCRT:std_type_info_static.obj
 0001:00008648       __isa_available_init       0000000140009648 f   MSVCRT:cpu_disp.obj
 0001:00008914       __scrt_is_ucrt_dll_in_use  0000000140009914 f   MSVCRT:ucrt_detection.obj
 0001:00008920       memcpy                     0000000140009920 f   vcruntime:VCRUNTIME140.dll
 0001:00008926       memset                     0000000140009926 f   vcruntime:VCRUNTIME140.dll
 0001:0000892c       __CxxFrameHandler4         000000014000992c f   vcruntime:VCRUNTIME140_1.dll
 0001:00008932       __C_specific_handler       0000000140009932 f   vcruntime:VCRUNTIME140.dll
 0001:00008938       __std_exception_copy       0000000140009938 f   vcruntime:VCRUNTIME140.dll
 0001:0000893e       __std_exception_destroy    000000014000993e f   vcruntime:VCRUNTIME140.dll
 0001:00008944       _CxxThrowException         0000000140009944 f   vcruntime:VCRUNTIME140.dll
 0001:0000894a       __current_exception        000000014000994a f   vcruntime:VCRUNTIME140.dll
 0001:00008950       __current_exception_context 0000000140009950 f   vcruntime:VCRUNTIME140.dll
 0001:00008956       strlen                     0000000140009956 f   ucrt:api-ms-win-crt-string-l1-1-0.dll
 0001:0000895c       strcpy                     000000014000995c f   ucrt:api-ms-win-crt-string-l1-1-0.dll
 0001:00008962       strcmp                     0000000140009962 f   ucrt:api-ms-win-crt-string-l1-1-0.dll
 0001:00008968       _callnewh                  0000000140009968 f   ucrt:api-ms-win-crt-heap-l1-1-0.dll
 0001:0000896e       malloc                     000000014000996e f   ucrt:api-ms-win-crt-heap-l1-1-0.dll
 0001:00008974       _seh_filter_exe            0000000140009974 f   ucrt:api-ms-win-crt-runtime-l1-1-0.dll
 0001:0000897a       _set_app_type              000000014000997a f   ucrt:api-ms-win-crt-runtime-l1-1-0.dll
 0001:00008980       __setusermatherr           0000000140009980 f   ucrt:api-ms-win-crt-math-l1-1-0.dll
 0001:00008986       _configure_narrow_argv     0000000140009986 f   ucrt:api-ms-win-crt-runtime-l1-1-0.dll
 0001:0000898c       _initialize_narrow_environment 000000014000998c f   ucrt:api-ms-win-crt-runtime-l1-1-0.dll
 0001:00008992       _get_narrow_winmain_command_line 0000000140009992 f   ucrt:api-ms-win-crt-runtime-l1-1-0.dll
 0001:00008998       _initterm                  0000000140009998 f   ucrt:api-ms-win-crt-runtime-l1-1-0.dll
 0001:0000899e       _initterm_e                000000014000999e f   ucrt:api-ms-win-crt-runtime-l1-1-0.dll
 0001:000089a4       exit                       00000001400099a4 f   ucrt:api-ms-win-crt-runtime-l1-1-0.dll
 0001:000089aa       _exit                      00000001400099aa f   ucrt:api-ms-win-crt-runtime-l1-1-0.dll
 0001:000089b0       _set_fmode                 00000001400099b0 f   ucrt:api-ms-win-crt-stdio-l1-1-0.dll
 0001:000089b6       _cexit                     00000001400099b6 f   ucrt:api-ms-win-crt-runtime-l1-1-0.dll
 0001:000089bc       _c_exit                    00000001400099bc f   ucrt:api-ms-win-crt-runtime-l1-1-0.dll
 0001:000089c2       _register_thread_local_exe_atexit_callback 00000001400099c2 f   ucrt:api-ms-win-crt-runtime-l1-1-0.dll
 0001:000089c8       _configthreadlocale        00000001400099c8 f   ucrt:api-ms-win-crt-locale-l1-1-0.dll
 0001:000089ce       _set_new_mode              00000001400099ce f   ucrt:api-ms-win-crt-heap-l1-1-0.dll
 0001:000089d4       __p__commode               00000001400099d4 f   ucrt:api-ms-win-crt-stdio-l1-1-0.dll
 0001:000089da       free                       00000001400099da f   ucrt:api-ms-win-crt-heap-l1-1-0.dll
 0001:000089e0       _initialize_onexit_table   00000001400099e0 f   ucrt:api-ms-win-crt-runtime-l1-1-0.dll
 0001:000089e6       _register_onexit_function  00000001400099e6 f   ucrt:api-ms-win-crt-runtime-l1-1-0.dll
 0001:000089ec       _crt_atexit                00000001400099ec f   ucrt:api-ms-win-crt-runtime-l1-1-0.dll
 0001:000089f2       terminate                  00000001400099f2 f   ucrt:api-ms-win-crt-runtime-l1-1-0.dll
 0001:00008a10       _guard_dispatch_icall_nop  0000000140009a10 f   MSVCRT:guard_dispatch.obj
 0001:00008a30       _guard_xfg_dispatch_icall_nop 0000000140009a30 f   MSVCRT:guard_xfg_dispatch.obj
 0002:00000000       __imp_InitCommonControlsEx 000000014000a000     comctl32:COMCTL32.dll
 0002:00000008       \177COMCTL32_NULL_THUNK_DATA 000000014000a008     comctl32:COMCTL32.dll
 0002:00000010       __imp_GetStockObject       000000014000a010     gdi32:GDI32.dll
 0002:00000018       \177GDI32_NULL_THUNK_DATA  000000014000a018     gdi32:GDI32.dll
 0002:00000020       __imp_GetModuleHandleW     000000014000a020     kernel32:KERNEL32.dll
 0002:00000028       __imp_GetStartupInfoW      000000014000a028     kernel32:KERNEL32.dll
 0002:00000030       __imp_IsDebuggerPresent    000000014000a030     kernel32:KERNEL32.dll
 0002:00000038       __imp_InitializeSListHead  000000014000a038     kernel32:KERNEL32.dll
 0002:00000040       __imp_GetCurrentThreadId   000000014000a040     kernel32:KERNEL32.dll
 0002:00000048       __imp_GetCurrentProcessId  000000014000a048     kernel32:KERNEL32.dll
 0002:00000050       __imp_QueryPerformanceCounter 000000014000a050     kernel32:KERNEL32.dll
 0002:00000058       __imp_IsProcessorFeaturePresent 000000014000a058     kernel32:KERNEL32.dll
 0002:00000060       __imp_TerminateProcess     000000014000a060     kernel32:KERNEL32.dll
 0002:00000068       __imp_GetCurrentProcess    000000014000a068     kernel32:KERNEL32.dll
 0002:00000070       __imp_SetUnhandledExceptionFilter 000000014000a070     kernel32:KERNEL32.dll
 0002:00000078       __imp_UnhandledExceptionFilter 000000014000a078     kernel32:KERNEL32.dll
 0002:00000080       __imp_RtlVirtualUnwind     000000014000a080     kernel32:KERNEL32.dll
 0002:00000088       __imp_RtlLookupFunctionEntry 000000014000a088     kernel32:KERNEL32.dll
 0002:00000090       __imp_RtlCaptureContext    000000014000a090     kernel32:KERNEL32.dll
 0002:00000098       __imp_FormatMessageA       000000014000a098     kernel32:KERNEL32.dll
 0002:000000a0       __imp_LocalFree            000000014000a0a0     kernel32:KERNEL32.dll
 0002:000000a8       __imp_GetSystemTimeAsFileTime 000000014000a0a8     kernel32:KERNEL32.dll
 0002:000000b0       __imp_LoadLibraryA         000000014000a0b0     kernel32:KERNEL32.dll
 0002:000000b8       __imp_GetProcAddress       000000014000a0b8     kernel32:KERNEL32.dll
 0002:000000c0       __imp_FreeLibrary          000000014000a0c0     kernel32:KERNEL32.dll
 0002:000000c8       __imp_GetLastError         000000014000a0c8     kernel32:KERNEL32.dll
 0002:000000d0       \177KERNEL32_NULL_THUNK_DATA 000000014000a0d0     kernel32:KERNEL32.dll
 0002:000000d8       __imp_EnumChildWindows     000000014000a0d8     user32:USER32.dll
 0002:000000e0       __imp_ScreenToClient       000000014000a0e0     user32:USER32.dll
 0002:000000e8       __imp_GetClassNameA        000000014000a0e8     user32:USER32.dll
 0002:000000f0       __imp_LoadCursorA          000000014000a0f0     user32:USER32.dll
 0002:000000f8       __imp_LoadIconA            000000014000a0f8     user32:USER32.dll
 0002:00000100       __imp_RegisterWindowMessageA 000000014000a100     user32:USER32.dll
 0002:00000108       __imp_GetCursorPos         000000014000a108     user32:USER32.dll
 0002:00000110       __imp_GetClientRect        000000014000a110     user32:USER32.dll
 0002:00000118       __imp_UpdateWindow         000000014000a118     user32:USER32.dll
 0002:00000120       __imp_TrackPopupMenu       000000014000a120     user32:USER32.dll
 0002:00000128       __imp_GetSubMenu           000000014000a128     user32:USER32.dll
 0002:00000130       __imp_LoadMenuA            000000014000a130     user32:USER32.dll
 0002:00000138       __imp_GetDlgItem           000000014000a138     user32:USER32.dll
 0002:00000140       __imp_EndDialog            000000014000a140     user32:USER32.dll
 0002:00000148       __imp_SetWindowPos         000000014000a148     user32:USER32.dll
 0002:00000150       __imp_ShowWindow           000000014000a150     user32:USER32.dll
 0002:00000158       __imp_DestroyWindow        000000014000a158     user32:USER32.dll
 0002:00000160       __imp_CreateWindowExA      000000014000a160     user32:USER32.dll
 0002:00000168       __imp_RegisterClassExA     000000014000a168     user32:USER32.dll
 0002:00000170       __imp_PostQuitMessage      000000014000a170     user32:USER32.dll
 0002:00000178       __imp_DefWindowProcA       000000014000a178     user32:USER32.dll
 0002:00000180       __imp_SendMessageA         000000014000a180     user32:USER32.dll
 0002:00000188       __imp_DispatchMessageA     000000014000a188     user32:USER32.dll
 0002:00000190       __imp_TranslateMessage     000000014000a190     user32:USER32.dll
 0002:00000198       __imp_GetMessageA          000000014000a198     user32:USER32.dll
 0002:000001a0       __imp_wsprintfA            000000014000a1a0     user32:USER32.dll
 0002:000001a8       __imp_SetDlgItemTextA      000000014000a1a8     user32:USER32.dll
 0002:000001b0       __imp_EnumWindows          000000014000a1b0     user32:USER32.dll
 0002:000001b8       \177USER32_NULL_THUNK_DATA 000000014000a1b8     user32:USER32.dll
 0002:000001c0       __imp_memcpy               000000014000a1c0     vcruntime:VCRUNTIME140.dll
 0002:000001c8       __imp_memset               000000014000a1c8     vcruntime:VCRUNTIME140.dll
 0002:000001d0       __imp___current_exception_context 000000014000a1d0     vcruntime:VCRUNTIME140.dll
 0002:000001d8       __imp___C_specific_handler 000000014000a1d8     vcruntime:VCRUNTIME140.dll
 0002:000001e0       __imp___std_exception_copy 000000014000a1e0     vcruntime:VCRUNTIME140.dll
 0002:000001e8       __imp___std_exception_destroy 000000014000a1e8     vcruntime:VCRUNTIME140.dll
 0002:000001f0       __imp__CxxThrowException   000000014000a1f0     vcruntime:VCRUNTIME140.dll
 0002:000001f8       __imp___current_exception  000000014000a1f8     vcruntime:VCRUNTIME140.dll
 0002:00000200       \177VCRUNTIME140_NULL_THUNK_DATA 000000014000a200     vcruntime:VCRUNTIME140.dll
 0002:00000208       __imp___CxxFrameHandler4   000000014000a208     vcruntime:VCRUNTIME140_1.dll
 0002:00000210       \177VCRUNTIME140_1_NULL_THUNK_DATA 000000014000a210     vcruntime:VCRUNTIME140_1.dll
 0002:00000218       __imp_getenv               000000014000a218     ucrt:api-ms-win-crt-environment-l1-1-0.dll
 0002:00000220       \177api-ms-win-crt-environment-l1-1-0_NULL_THUNK_DATA 000000014000a220     ucrt:api-ms-win-crt-environment-l1-1-0.dll
 0002:00000228       __imp_malloc               000000014000a228     ucrt:api-ms-win-crt-heap-l1-1-0.dll
 0002:00000230       __imp__callnewh            000000014000a230     ucrt:api-ms-win-crt-heap-l1-1-0.dll
 0002:00000238       __imp__set_new_mode        000000014000a238     ucrt:api-ms-win-crt-heap-l1-1-0.dll
 0002:00000240       __imp_free                 000000014000a240     ucrt:api-ms-win-crt-heap-l1-1-0.dll
 0002:00000248       \177api-ms-win-crt-heap-l1-1-0_NULL_THUNK_DATA 000000014000a248     ucrt:api-ms-win-crt-heap-l1-1-0.dll
 0002:00000250       __imp__configthreadlocale  000000014000a250     ucrt:api-ms-win-crt-locale-l1-1-0.dll
 0002:00000258       \177api-ms-win-crt-locale-l1-1-0_NULL_THUNK_DATA 000000014000a258     ucrt:api-ms-win-crt-locale-l1-1-0.dll
 0002:00000260       __imp___setusermatherr     000000014000a260     ucrt:api-ms-win-crt-math-l1-1-0.dll
 0002:00000268       \177api-ms-win-crt-math-l1-1-0_NULL_THUNK_DATA 000000014000a268     ucrt:api-ms-win-crt-math-l1-1-0.dll
 0002:00000270       __imp_terminate            000000014000a270     ucrt:api-ms-win-crt-runtime-l1-1-0.dll
 0002:00000278       __imp__crt_atexit          000000014000a278     ucrt:api-ms-win-crt-runtime-l1-1-0.dll
 0002:00000280       __imp__register_onexit_function 000000014000a280     ucrt:api-ms-win-crt-runtime-l1-1-0.dll
 0002:00000288       __imp__initialize_onexit_table 000000014000a288     ucrt:api-ms-win-crt-runtime-l1-1-0.dll
 0002:00000290       __imp__register_thread_local_exe_atexit_callback 000000014000a290     ucrt:api-ms-win-crt-runtime-l1-1-0.dll
 0002:00000298       __imp__seh_filter_exe      000000014000a298     ucrt:api-ms-win-crt-runtime-l1-1-0.dll
 0002:000002a0       __imp__set_app_type        000000014000a2a0     ucrt:api-ms-win-crt-runtime-l1-1-0.dll
 0002:000002a8       __imp__cexit               000000014000a2a8     ucrt:api-ms-win-crt-runtime-l1-1-0.dll
 0002:000002b0       __imp__configure_narrow_argv 000000014000a2b0     ucrt:api-ms-win-crt-runtime-l1-1-0.dll
 0002:000002b8       __imp__initialize_narrow_environment 000000014000a2b8     ucrt:api-ms-win-crt-runtime-l1-1-0.dll
 0002:000002c0       __imp__c_exit              000000014000a2c0     ucrt:api-ms-win-crt-runtime-l1-1-0.dll
 0002:000002c8       __imp__initterm            000000014000a2c8     ucrt:api-ms-win-crt-runtime-l1-1-0.dll
 0002:000002d0       __imp__initterm_e          000000014000a2d0     ucrt:api-ms-win-crt-runtime-l1-1-0.dll
 0002:000002d8       __imp_exit                 000000014000a2d8     ucrt:api-ms-win-crt-runtime-l1-1-0.dll
 0002:000002e0       __imp__exit                000000014000a2e0     ucrt:api-ms-win-crt-runtime-l1-1-0.dll
 0002:000002e8       __imp__get_narrow_winmain_command_line 000000014000a2e8     ucrt:api-ms-win-crt-runtime-l1-1-0.dll
 0002:000002f0       \177api-ms-win-crt-runtime-l1-1-0_NULL_THUNK_DATA 000000014000a2f0     ucrt:api-ms-win-crt-runtime-l1-1-0.dll
 0002:000002f8       __imp_fclose               000000014000a2f8     ucrt:api-ms-win-crt-stdio-l1-1-0.dll
 0002:00000300       __imp_fopen                000000014000a300     ucrt:api-ms-win-crt-stdio-l1-1-0.dll
 0002:00000308       __imp___stdio_common_vfwprintf 000000014000a308     ucrt:api-ms-win-crt-stdio-l1-1-0.dll
 0002:00000310       __imp___acrt_iob_func      000000014000a310     ucrt:api-ms-win-crt-stdio-l1-1-0.dll
 0002:00000318       __imp___p__commode         000000014000a318     ucrt:api-ms-win-crt-stdio-l1-1-0.dll
 0002:00000320       __imp___stdio_common_vsprintf 000000014000a320     ucrt:api-ms-win-crt-stdio-l1-1-0.dll
 0002:00000328       __imp___stdio_common_vfprintf 000000014000a328     ucrt:api-ms-win-crt-stdio-l1-1-0.dll
 0002:00000330       __imp__set_fmode           000000014000a330     ucrt:api-ms-win-crt-stdio-l1-1-0.dll
 0002:00000338       __imp_fflush               000000014000a338     ucrt:api-ms-win-crt-stdio-l1-1-0.dll
 0002:00000340       \177api-ms-win-crt-stdio-l1-1-0_NULL_THUNK_DATA 000000014000a340     ucrt:api-ms-win-crt-stdio-l1-1-0.dll
 0002:00000348       __imp_wcscmp               000000014000a348     ucrt:api-ms-win-crt-string-l1-1-0.dll
 0002:00000350       __imp_strncpy              000000014000a350     ucrt:api-ms-win-crt-string-l1-1-0.dll
 0002:00000358       __imp_strlen               000000014000a358     ucrt:api-ms-win-crt-string-l1-1-0.dll
 0002:00000360       __imp_strcmp               000000014000a360     ucrt:api-ms-win-crt-string-l1-1-0.dll
 0002:00000368       __imp_strcpy               000000014000a368     ucrt:api-ms-win-crt-string-l1-1-0.dll
 0002:00000370       __imp_strncat              000000014000a370     ucrt:api-ms-win-crt-string-l1-1-0.dll
 0002:00000378       \177api-ms-win-crt-string-l1-1-0_NULL_THUNK_DATA 000000014000a378     ucrt:api-ms-win-crt-string-l1-1-0.dll
 0002:00000380       __imp_asctime              000000014000a380     ucrt:api-ms-win-crt-time-l1-1-0.dll
 0002:00000388       __imp__time64              000000014000a388     ucrt:api-ms-win-crt-time-l1-1-0.dll
 0002:00000390       __imp__localtime64         000000014000a390     ucrt:api-ms-win-crt-time-l1-1-0.dll
 0002:00000398       \177api-ms-win-crt-time-l1-1-0_NULL_THUNK_DATA 000000014000a398     ucrt:api-ms-win-crt-time-l1-1-0.dll
 0002:000003a0       __guard_check_icall_fptr   000000014000a3a0     MSVCRT:guard_support.obj
 0002:000003a8       __guard_xfg_check_icall_fptr 000000014000a3a8     MSVCRT:guard_support.obj
 0002:000003b0       __guard_dispatch_icall_fptr 000000014000a3b0     MSVCRT:guard_support.obj
 0002:000003b8       __guard_xfg_dispatch_icall_fptr 000000014000a3b8     MSVCRT:guard_support.obj
 0002:000003c0       __guard_xfg_table_dispatch_icall_fptr 000000014000a3c0     MSVCRT:guard_support.obj
 0002:000003c8       __castguard_check_failure_os_handled_fptr 000000014000a3c8     MSVCRT:guard_support.obj
 0002:000003d0       __guard_memcpy_fptr        000000014000a3d0     vcruntime:softmemtag.obj
 0002:000003d8       __xc_a                     000000014000a3d8     MSVCRT:initializers.obj
 0002:000003e8       __xc_z                     000000014000a3e8     MSVCRT:initializers.obj
 0002:000003f0       __xi_a                     000000014000a3f0     MSVCRT:initializers.obj
 0002:00000408       __xi_z                     000000014000a408     MSVCRT:initializers.obj
 0002:00000410       __xp_a                     000000014000a410     MSVCRT:initializers.obj
 0002:00000418       __xp_z                     000000014000a418     MSVCRT:initializers.obj
 0002:00000420       __xt_a                     000000014000a420     MSVCRT:initializers.obj
 0002:00000428       __xt_z                     000000014000a428     MSVCRT:initializers.obj
 0002:00001ee0       ??_7exception@std@@6B@     000000014000bee0     MSVCRT:throw_bad_alloc.obj
 0002:00001ef0       ??_C@_0BC@EOODALEL@Unknown?5exception@ 000000014000bef0     MSVCRT:throw_bad_alloc.obj
 0002:00001f10       ??_7bad_alloc@std@@6B@     000000014000bf10     MSVCRT:throw_bad_alloc.obj
 0002:00001f20       ??_C@_0P@GHFPNOJB@bad?5allocation@ 000000014000bf20     MSVCRT:throw_bad_alloc.obj
 0002:00001f38       ??_7bad_array_new_length@std@@6B@ 000000014000bf38     MSVCRT:throw_bad_alloc.obj
 0002:00001f48       ??_C@_0BF@KINCDENJ@bad?5array?5new?5length@ 000000014000bf48     MSVCRT:throw_bad_alloc.obj
 0002:00001f60       __xmm@ffffffffffffffffffffffffffffffff 000000014000bf60     MSVCRT:utility.obj
 0002:00001f78       ??_7type_info@@6B@         000000014000bf78     MSVCRT:std_type_info_static.obj
 0002:00001f80       _load_config_used          000000014000bf80     MSVCRT:loadcfg.obj
 0002:00002180       ??_R4exception@std@@6B@    000000014000c180     MSVCRT:throw_bad_alloc.obj
 0002:000021a8       ??_R3exception@std@@8      000000014000c1a8     MSVCRT:throw_bad_alloc.obj
 0002:000021c0       ??_R2exception@std@@8      000000014000c1c0     MSVCRT:throw_bad_alloc.obj
 0002:000021d0       ??_R1A@?0A@EA@exception@std@@8 000000014000c1d0     MSVCRT:throw_bad_alloc.obj
 0002:000021f8       ??_R4bad_array_new_length@std@@6B@ 000000014000c1f8     MSVCRT:throw_bad_alloc.obj
 0002:00002220       ??_R3bad_array_new_length@std@@8 000000014000c220     MSVCRT:throw_bad_alloc.obj
 0002:00002238       ??_R2bad_array_new_length@std@@8 000000014000c238     MSVCRT:throw_bad_alloc.obj
 0002:00002258       ??_R1A@?0A@EA@bad_array_new_length@std@@8 000000014000c258     MSVCRT:throw_bad_alloc.obj
 0002:00002280       ??_R1A@?0A@EA@bad_alloc@std@@8 000000014000c280     MSVCRT:throw_bad_alloc.obj
 0002:000022a8       ??_R3bad_alloc@std@@8      000000014000c2a8     MSVCRT:throw_bad_alloc.obj
 0002:000022c0       ??_R2bad_alloc@std@@8      000000014000c2c0     MSVCRT:throw_bad_alloc.obj
 0002:000022d8       ??_R4bad_alloc@std@@6B@    000000014000c2d8     MSVCRT:throw_bad_alloc.obj
 0002:00002300       ??_R4type_info@@6B@        000000014000c300     MSVCRT:std_type_info_static.obj
 0002:00002328       ??_R3type_info@@8          000000014000c328     MSVCRT:std_type_info_static.obj
 0002:00002340       ??_R2type_info@@8          000000014000c340     MSVCRT:std_type_info_static.obj
 0002:00002350       ??_R1A@?0A@EA@type_info@@8 000000014000c350     MSVCRT:std_type_info_static.obj
 0002:00002374       __volatile_metadata        000000014000c374     <linker-defined>
 0002:00002768       __rtc_iaa                  000000014000c768     MSVCRT:initsect.obj
 0002:00002770       __rtc_izz                  000000014000c770     MSVCRT:initsect.obj
 0002:00002778       __rtc_taa                  000000014000c778     MSVCRT:initsect.obj
 0002:00002780       __rtc_tzz                  000000014000c780     MSVCRT:initsect.obj
 0002:00002d50       _TI2?AVbad_alloc@std@@     000000014000cd50     MSVCRT:throw_bad_alloc.obj
 0002:00002d70       _CTA2?AVbad_alloc@std@@    000000014000cd70     MSVCRT:throw_bad_alloc.obj
 0002:00002d88       _CT??_R0?AVbad_alloc@std@@@8??0bad_alloc@std@@QEAA@AEBV01@@Z24 000000014000cd88     MSVCRT:throw_bad_alloc.obj
 0002:00002db0       _CT??_R0?AVexception@std@@@8??0exception@std@@QEAA@AEBV01@@Z24 000000014000cdb0     MSVCRT:throw_bad_alloc.obj
 0002:00002dd8       _TI3?AVbad_array_new_length@std@@ 000000014000cdd8     MSVCRT:throw_bad_alloc.obj
 0002:00002df8       _CTA3?AVbad_array_new_length@std@@ 000000014000cdf8     MSVCRT:throw_bad_alloc.obj
 0002:00002e18       _CT??_R0?AVbad_array_new_length@std@@@8??0bad_array_new_length@std@@QEAA@AEBV01@@Z24 000000014000ce18     MSVCRT:throw_bad_alloc.obj
 0002:00002e3c       __IMPORT_DESCRIPTOR_COMCTL32 000000014000ce3c     comctl32:COMCTL32.dll
 0002:00002e50       __IMPORT_DESCRIPTOR_GDI32  000000014000ce50     gdi32:GDI32.dll
 0002:00002e64       __IMPORT_DESCRIPTOR_USER32 000000014000ce64     user32:USER32.dll
 0002:00002e78       __IMPORT_DESCRIPTOR_KERNEL32 000000014000ce78     kernel32:KERNEL32.dll
 0002:00002e8c       __IMPORT_DESCRIPTOR_VCRUNTIME140 000000014000ce8c     vcruntime:VCRUNTIME140.dll
 0002:00002ea0       __IMPORT_DESCRIPTOR_VCRUNTIME140_1 000000014000cea0     vcruntime:VCRUNTIME140_1.dll
 0002:00002eb4       __IMPORT_DESCRIPTOR_api-ms-win-crt-string-l1-1-0 000000014000ceb4     ucrt:api-ms-win-crt-string-l1-1-0.dll
 0002:00002ec8       __IMPORT_DESCRIPTOR_api-ms-win-crt-stdio-l1-1-0 000000014000cec8     ucrt:api-ms-win-crt-stdio-l1-1-0.dll
 0002:00002edc       __IMPORT_DESCRIPTOR_api-ms-win-crt-environment-l1-1-0 000000014000cedc     ucrt:api-ms-win-crt-environment-l1-1-0.dll
 0002:00002ef0       __IMPORT_DESCRIPTOR_api-ms-win-crt-time-l1-1-0 000000014000cef0     ucrt:api-ms-win-crt-time-l1-1-0.dll
 0002:00002f04       __IMPORT_DESCRIPTOR_api-ms-win-crt-heap-l1-1-0 000000014000cf04     ucrt:api-ms-win-crt-heap-l1-1-0.dll
 0002:00002f18       __IMPORT_DESCRIPTOR_api-ms-win-crt-runtime-l1-1-0 000000014000cf18     ucrt:api-ms-win-crt-runtime-l1-1-0.dll
 0002:00002f2c       __IMPORT_DESCRIPTOR_api-ms-win-crt-math-l1-1-0 000000014000cf2c     ucrt:api-ms-win-crt-math-l1-1-0.dll
 0002:00002f40       __IMPORT_DESCRIPTOR_api-ms-win-crt-locale-l1-1-0 000000014000cf40     ucrt:api-ms-win-crt-locale-l1-1-0.dll
 0002:00002f54       __NULL_IMPORT_DESCRIPTOR   000000014000cf54     comctl32:COMCTL32.dll
 0003:00000b30       ?depth@@3HA                000000014000eb30     jaccesswalker.obj
 0003:00000b38       ?theJaccesswalkerClassName@@3PADA 000000014000eb38     jaccesswalker.obj
 0003:00000b50       ?theAccessInfoClassName@@3PADA 000000014000eb50     jaccesswalker.obj
 0003:00000bc0       __security_cookie          000000014000ebc0     MSVCRT:gs_cookie.obj
 0003:00000c00       __security_cookie_complement 000000014000ec00     MSVCRT:gs_cookie.obj
 0003:00000c08       _fltused                   000000014000ec08     MSVCRT:fltused.obj
 0003:00000c0c       __scrt_native_dllmain_reason 000000014000ec0c     MSVCRT:utility.obj
 0003:00000c10       __scrt_default_matherr     000000014000ec10     MSVCRT:matherr.obj
 0003:00000c18       __isa_inverted             000000014000ec18     MSVCRT:cpu_disp.obj
 0003:00000c20       __isa_available            000000014000ec20     MSVCRT:cpu_disp.obj
 0003:00000c24       __isa_enabled              000000014000ec24     MSVCRT:cpu_disp.obj
 0003:00000c28       __memset_fast_string_threshold 000000014000ec28     MSVCRT:cpu_disp.obj
 0003:00000c30       __memset_nt_threshold      000000014000ec30     MSVCRT:cpu_disp.obj
 0003:00000c40       __scrt_ucrt_dll_is_in_use  000000014000ec40     MSVCRT:ucrt_stubs.obj
 0003:00000c48       ??_R0?AVbad_alloc@std@@@8  000000014000ec48     MSVCRT:throw_bad_alloc.obj
 0003:00000c70       ??_R0?AVexception@std@@@8  000000014000ec70     MSVCRT:throw_bad_alloc.obj
 0003:00000c98       ??_R0?AVbad_array_new_length@std@@@8 000000014000ec98     MSVCRT:throw_bad_alloc.obj
 0003:00000cc8       ??_R0?AVtype_info@@@8      000000014000ecc8     MSVCRT:std_type_info_static.obj
 0003:00000d00       theAccessBridgeInitializedFlag 000000014000ed00     AccessBridgeCalls.obj
 0003:00000d08       ?_OptionsStorage@?1??__local_stdio_printf_options@@9@4_KA 000000014000ed08     AccessBridgeDebug.obj
 0003:00000e20       ?theFromJavaHelloMsgID@@3IA 000000014000ee20     AccessBridgeMessages.obj
 0003:00000e24       ?theFromWindowsHelloMsgID@@3IA 000000014000ee24     AccessBridgeMessages.obj
 0003:00000e28       ?g_LogStringCallback@@3P6AXPEBD@ZEA 000000014000ee28     AccessInfo.obj
 0003:00000e70       ?ourHwnd@@3PEAUHWND__@@EA  000000014000ee70     jaccesswalker.obj
 0003:00000e78       ?topLevelWindow@@3PEAUHWND__@@EA 000000014000ee78     jaccesswalker.obj
 0003:00000e80       ?logfile@@3PEAU_iobuf@@EA  000000014000ee80     jaccesswalker.obj
 0003:00000e88       ?popupMenu@@3PEAUHMENU__@@EA 000000014000ee88     jaccesswalker.obj
 0003:00000e90       ?theJaccesswalkerWindow@@3PEAUHWND__@@EA 000000014000ee90     jaccesswalker.obj
 0003:00000e98       ?theTreeControlWindow@@3PEAUHWND__@@EA 000000014000ee98     jaccesswalker.obj
 0003:00000ea0       ?theInstance@@3PEAUHINSTANCE__@@EA 000000014000eea0     jaccesswalker.obj
 0003:00000ea8       ?theJaccesswalker@@3PEAVJaccesswalker@@EA 000000014000eea8     jaccesswalker.obj
 0003:00000eb0       ?theSelectedNode@@3PEAVAccessibleNode@@EA 000000014000eeb0     jaccesswalker.obj
 0003:00000eb8       ?thePopupNode@@3PEAVAccessibleNode@@EA 000000014000eeb8     jaccesswalker.obj
 0003:00000ec0       ?theSelectedAccessibleContext@@3_JA 000000014000eec0     jaccesswalker.obj
 0003:00000ec8       ?hwndTV@@3PEAUHWND__@@EA   000000014000eec8     jaccesswalker.obj
 0003:00001440       __scrt_current_native_startup_state 000000014000f440     MSVCRT:utility.obj
 0003:00001448       __scrt_native_startup_lock 000000014000f448     MSVCRT:utility.obj
 0003:00001490       ?__type_info_root_node@@3U__type_info_node@@A 000000014000f490     MSVCRT:tncleanup.obj
 0003:000014a0       ?_OptionsStorage@?1??__local_stdio_scanf_options@@9@4_KA 000000014000f4a0     MSVCRT:default_local_stdio_options.obj
 0003:000014a8       __scrt_debugger_hook_flag  000000014000f4a8     MSVCRT:utility_desktop.obj
 0003:000014ac       __avx10_version            000000014000f4ac     MSVCRT:cpu_disp.obj
 0003:000014b0       __favor                    000000014000f4b0     MSVCRT:cpu_disp.obj
 0003:000014c0       theAccessBridge            000000014000f4c0     <common>
 0003:000017c8       theAccessBridgeInstance    000000014000f7c8     <common>
 0003:000017d0       __dyn_tls_dtor_callback    000000014000f7d0     <common>
 0003:000017d8       __dyn_tls_init_callback    000000014000f7d8     <common>

 entry point at        0001:00007e44

 Static symbols

 0000:fffed000       .debug$S                   0000000140000000     vcruntime:VCRUNTIME140.dll
 0000:fffed000       .debug$S                   0000000140000000     vcruntime:VCRUNTIME140.dll
 0000:fffed000       .debug$S                   0000000140000000     vcruntime:VCRUNTIME140.dll
 0000:fffed000       .debug$S                   0000000140000000     vcruntime:VCRUNTIME140.dll
 0000:fffed000       .debug$S                   0000000140000000     vcruntime:VCRUNTIME140.dll
 0000:fffed000       .debug$S                   0000000140000000     vcruntime:VCRUNTIME140.dll
 0000:fffed000       .debug$S                   0000000140000000     vcruntime:VCRUNTIME140.dll
 0000:fffed000       .debug$S                   0000000140000000     vcruntime:VCRUNTIME140.dll
 0000:fffed000       .debug$S                   0000000140000000     vcruntime:VCRUNTIME140.dll
 0000:fffed000       .debug$S                   0000000140000000     vcruntime:VCRUNTIME140_1.dll
 0000:fffed000       .debug$S                   0000000140000000     ucrt:api-ms-win-crt-environment-l1-1-0.dll
 0000:fffed000       .debug$S                   0000000140000000     ucrt:api-ms-win-crt-heap-l1-1-0.dll
 0000:fffed000       .debug$S                   0000000140000000     ucrt:api-ms-win-crt-heap-l1-1-0.dll
 0000:fffed000       .debug$S                   0000000140000000     ucrt:api-ms-win-crt-heap-l1-1-0.dll
 0000:fffed000       .debug$S                   0000000140000000     ucrt:api-ms-win-crt-heap-l1-1-0.dll
 0000:fffed000       .debug$S                   0000000140000000     ucrt:api-ms-win-crt-locale-l1-1-0.dll
 0000:fffed000       .debug$S                   0000000140000000     ucrt:api-ms-win-crt-math-l1-1-0.dll
 0000:fffed000       .debug$S                   0000000140000000     ucrt:api-ms-win-crt-runtime-l1-1-0.dll
 0000:fffed000       .debug$S                   0000000140000000     ucrt:api-ms-win-crt-runtime-l1-1-0.dll
 0000:fffed000       .debug$S                   0000000140000000     ucrt:api-ms-win-crt-runtime-l1-1-0.dll
 0000:fffed000       .debug$S                   0000000140000000     ucrt:api-ms-win-crt-runtime-l1-1-0.dll
 0000:fffed000       .debug$S                   0000000140000000     ucrt:api-ms-win-crt-runtime-l1-1-0.dll
 0000:fffed000       .debug$S                   0000000140000000     ucrt:api-ms-win-crt-runtime-l1-1-0.dll
 0000:fffed000       .debug$S                   0000000140000000     ucrt:api-ms-win-crt-runtime-l1-1-0.dll
 0000:fffed000       .debug$S                   0000000140000000     ucrt:api-ms-win-crt-runtime-l1-1-0.dll
 0000:fffed000       .debug$S                   0000000140000000     ucrt:api-ms-win-crt-runtime-l1-1-0.dll
 0000:fffed000       .debug$S                   0000000140000000     ucrt:api-ms-win-crt-runtime-l1-1-0.dll
 0000:fffed000       .debug$S                   0000000140000000     ucrt:api-ms-win-crt-runtime-l1-1-0.dll
 0000:fffed000       .debug$S                   0000000140000000     ucrt:api-ms-win-crt-runtime-l1-1-0.dll
 0000:fffed000       .debug$S                   0000000140000000     ucrt:api-ms-win-crt-runtime-l1-1-0.dll
 0000:fffed000       .debug$S                   0000000140000000     ucrt:api-ms-win-crt-runtime-l1-1-0.dll
 0000:fffed000       .debug$S                   0000000140000000     ucrt:api-ms-win-crt-runtime-l1-1-0.dll
 0000:fffed000       .debug$S                   0000000140000000     ucrt:api-ms-win-crt-runtime-l1-1-0.dll
 0000:fffed000       .debug$S                   0000000140000000     ucrt:api-ms-win-crt-runtime-l1-1-0.dll
 0000:fffed000       .debug$S                   0000000140000000     ucrt:api-ms-win-crt-runtime-l1-1-0.dll
 0000:fffed000       .debug$S                   0000000140000000     ucrt:api-ms-win-crt-runtime-l1-1-0.dll
 0000:fffed000       .debug$S                   0000000140000000     ucrt:api-ms-win-crt-stdio-l1-1-0.dll
 0000:fffed000       .debug$S                   0000000140000000     ucrt:api-ms-win-crt-stdio-l1-1-0.dll
 0000:fffed000       .debug$S                   0000000140000000     ucrt:api-ms-win-crt-stdio-l1-1-0.dll
 0000:fffed000       .debug$S                   0000000140000000     ucrt:api-ms-win-crt-stdio-l1-1-0.dll
 0000:fffed000       .debug$S                   0000000140000000     ucrt:api-ms-win-crt-stdio-l1-1-0.dll
 0000:fffed000       .debug$S                   0000000140000000     ucrt:api-ms-win-crt-stdio-l1-1-0.dll
 0000:fffed000       .debug$S                   0000000140000000     ucrt:api-ms-win-crt-stdio-l1-1-0.dll
 0000:fffed000       .debug$S                   0000000140000000     ucrt:api-ms-win-crt-stdio-l1-1-0.dll
 0000:fffed000       .debug$S                   0000000140000000     ucrt:api-ms-win-crt-stdio-l1-1-0.dll
 0000:fffed000       .debug$S                   0000000140000000     ucrt:api-ms-win-crt-string-l1-1-0.dll
 0000:fffed000       .debug$S                   0000000140000000     ucrt:api-ms-win-crt-string-l1-1-0.dll
 0000:fffed000       .debug$S                   0000000140000000     ucrt:api-ms-win-crt-string-l1-1-0.dll
 0000:fffed000       .debug$S                   0000000140000000     ucrt:api-ms-win-crt-string-l1-1-0.dll
 0000:fffed000       .debug$S                   0000000140000000     ucrt:api-ms-win-crt-string-l1-1-0.dll
 0000:fffed000       .debug$S                   0000000140000000     ucrt:api-ms-win-crt-string-l1-1-0.dll
 0000:fffed000       .debug$S                   0000000140000000     ucrt:api-ms-win-crt-time-l1-1-0.dll
 0000:fffed000       .debug$S                   0000000140000000     ucrt:api-ms-win-crt-time-l1-1-0.dll
 0000:fffed000       .debug$S                   0000000140000000     ucrt:api-ms-win-crt-time-l1-1-0.dll
 0000:fffed000       .debug$S                   0000000140000000     comctl32:COMCTL32.dll
 0000:fffed000       .debug$S                   0000000140000000     gdi32:GDI32.dll
 0000:fffed000       .debug$S                   0000000140000000     kernel32:KERNEL32.dll
 0000:fffed000       .debug$S                   0000000140000000     kernel32:KERNEL32.dll
 0000:fffed000       .debug$S                   0000000140000000     kernel32:KERNEL32.dll
 0000:fffed000       .debug$S                   0000000140000000     kernel32:KERNEL32.dll
 0000:fffed000       .debug$S                   0000000140000000     kernel32:KERNEL32.dll
 0000:fffed000       .debug$S                   0000000140000000     kernel32:KERNEL32.dll
 0000:fffed000       .debug$S                   0000000140000000     kernel32:KERNEL32.dll
 0000:fffed000       .debug$S                   0000000140000000     kernel32:KERNEL32.dll
 0000:fffed000       .debug$S                   0000000140000000     kernel32:KERNEL32.dll
 0000:fffed000       .debug$S                   0000000140000000     kernel32:KERNEL32.dll
 0000:fffed000       .debug$S                   0000000140000000     kernel32:KERNEL32.dll
 0000:fffed000       .debug$S                   0000000140000000     kernel32:KERNEL32.dll
 0000:fffed000       .debug$S                   0000000140000000     kernel32:KERNEL32.dll
 0000:fffed000       .debug$S                   0000000140000000     kernel32:KERNEL32.dll
 0000:fffed000       .debug$S                   0000000140000000     kernel32:KERNEL32.dll
 0000:fffed000       .debug$S                   0000000140000000     kernel32:KERNEL32.dll
 0000:fffed000       .debug$S                   0000000140000000     kernel32:KERNEL32.dll
 0000:fffed000       .debug$S                   0000000140000000     kernel32:KERNEL32.dll
 0000:fffed000       .debug$S                   0000000140000000     kernel32:KERNEL32.dll
 0000:fffed000       .debug$S                   0000000140000000     kernel32:KERNEL32.dll
 0000:fffed000       .debug$S                   0000000140000000     kernel32:KERNEL32.dll
 0000:fffed000       .debug$S                   0000000140000000     kernel32:KERNEL32.dll
 0000:fffed000       .debug$S                   0000000140000000     user32:USER32.dll
 0000:fffed000       .debug$S                   0000000140000000     user32:USER32.dll
 0000:fffed000       .debug$S                   0000000140000000     user32:USER32.dll
 0000:fffed000       .debug$S                   0000000140000000     user32:USER32.dll
 0000:fffed000       .debug$S                   0000000140000000     user32:USER32.dll
 0000:fffed000       .debug$S                   0000000140000000     user32:USER32.dll
 0000:fffed000       .debug$S                   0000000140000000     user32:USER32.dll
 0000:fffed000       .debug$S                   0000000140000000     user32:USER32.dll
 0000:fffed000       .debug$S                   0000000140000000     user32:USER32.dll
 0000:fffed000       .debug$S                   0000000140000000     user32:USER32.dll
 0000:fffed000       .debug$S                   0000000140000000     user32:USER32.dll
 0000:fffed000       .debug$S                   0000000140000000     user32:USER32.dll
 0000:fffed000       .debug$S                   0000000140000000     user32:USER32.dll
 0000:fffed000       .debug$S                   0000000140000000     user32:USER32.dll
 0000:fffed000       .debug$S                   0000000140000000     user32:USER32.dll
 0000:fffed000       .debug$S                   0000000140000000     user32:USER32.dll
 0000:fffed000       .debug$S                   0000000140000000     user32:USER32.dll
 0000:fffed000       .debug$S                   0000000140000000     user32:USER32.dll
 0000:fffed000       .debug$S                   0000000140000000     user32:USER32.dll
 0000:fffed000       .debug$S                   0000000140000000     user32:USER32.dll
 0000:fffed000       .debug$S                   0000000140000000     user32:USER32.dll
 0000:fffed000       .debug$S                   0000000140000000     user32:USER32.dll
 0000:fffed000       .debug$S                   0000000140000000     user32:USER32.dll
 0000:fffed000       .debug$S                   0000000140000000     user32:USER32.dll
 0000:fffed000       .debug$S                   0000000140000000     user32:USER32.dll
 0000:fffed000       .debug$S                   0000000140000000     user32:USER32.dll
 0000:fffed000       .debug$S                   0000000140000000     user32:USER32.dll
 0000:fffed000       .debug$S                   0000000140000000     user32:USER32.dll
 0001:00005db0       localtime                  0000000140006db0 f   AccessInfo.obj
 0001:00005dd0       time                       0000000140006dd0 f   AccessInfo.obj
 0001:00007938       capture_current_context    0000000140008938 f   MSVCRT:gs_report.obj
 0001:000079a8       capture_previous_context   00000001400089a8 f   MSVCRT:gs_report.obj
 0001:00007aa0       $$000000                   0000000140008aa0     MSVCRT:chkstk.obj
 0001:00007b00       $$000000                   0000000140008b00     MSVCRT:amdsecgs.obj
 0001:00007bec       ?pre_c_initialization@@YAHXZ 0000000140008bec f   MSVCRT:exe_winmain.obj
 0001:00007ca4       ?post_pgo_initialization@@YAHXZ 0000000140008ca4 f   MSVCRT:exe_winmain.obj
 0001:00007cb4       ?pre_cpp_initialization@@YAXXZ 0000000140008cb4 f   MSVCRT:exe_winmain.obj
 0001:00007cd0       ?__scrt_common_main_seh@@YAHXZ 0000000140008cd0 f   MSVCRT:exe_winmain.obj
 0001:00008a00       $$000000                   0000000140009a00     MSVCRT:guard_dispatch.obj
 0001:00008a20       $$000000                   0000000140009a20     MSVCRT:guard_xfg_dispatch.obj
 0001:00008a40       ?dtor$0@?0??addComponentNodes@Jaccesswalker@@QEAAXJ_JPEAVAccessibleNode@@PEAUHWND__@@PEAU_TREEITEM@@2@Z@4HA 0000000140009a40 f   jaccesswalker.obj
 0001:00008a5d       ?filt$0@?0??__scrt_common_main_seh@@YAHXZ@4HA 0000000140009a5d f   MSVCRT:exe_winmain.obj
 0001:00008a7b       __scrt_is_nonwritable_in_current_image$filt$0 0000000140009a7b f   MSVCRT:utility.obj
 0002:000003e0       ?pre_cpp_initializer@@3P6AXXZEA 000000014000a3e0     MSVCRT:exe_winmain.obj
 0002:000003f8       ?pre_c_initializer@@3P6AHXZEA 000000014000a3f8     MSVCRT:exe_winmain.obj
 0002:00000400       ?post_pgo_initializer@@3P6AHXZEA 000000014000a400     MSVCRT:exe_winmain.obj
 0002:00000430       $SG43284                   000000014000a430     AccessBridgeDebug.obj
 0002:0000044c       $SG43286                   000000014000a44c     AccessBridgeDebug.obj
 0002:00000454       $SG43287                   000000014000a454     AccessBridgeDebug.obj
 0002:00000458       $SG43289                   000000014000a458     AccessBridgeDebug.obj
 0002:00000460       $SG43290                   000000014000a460     AccessBridgeDebug.obj
 0002:00000478       $SG43317                   000000014000a478     AccessBridgeDebug.obj
 0002:00000498       $SG43318                   000000014000a498     AccessBridgeDebug.obj
 0002:000004a4       $SG43320                   000000014000a4a4     AccessBridgeDebug.obj
 0002:000004a8       $SG43331                   000000014000a4a8     AccessBridgeDebug.obj
 0002:000004b0       $SG43332                   000000014000a4b0     AccessBridgeDebug.obj
 0002:000004b8       $SG43343                   000000014000a4b8     AccessBridgeDebug.obj
 0002:000004c0       $SG43344                   000000014000a4c0     AccessBridgeDebug.obj
 0002:000004c8       $SG43355                   000000014000a4c8     AccessBridgeDebug.obj
 0002:000004d0       $SG43356                   000000014000a4d0     AccessBridgeDebug.obj
 0002:000004d8       $SG43367                   000000014000a4d8     AccessBridgeDebug.obj
 0002:000004e0       $SG43368                   000000014000a4e0     AccessBridgeDebug.obj
 0002:000004e8       $SG38649                   000000014000a4e8     AccessBridgeMessages.obj
 0002:00000508       $SG38650                   000000014000a508     AccessBridgeMessages.obj
 0002:00000530       $SG47502                   000000014000a530     AccessInfo.obj
 0002:00000534       $SG47504                   000000014000a534     AccessInfo.obj
 0002:00000538       $SG47507                   000000014000a538     AccessInfo.obj
 0002:00000548       $SG47547                   000000014000a548     AccessInfo.obj
 0002:00000574       $SG47548                   000000014000a574     AccessInfo.obj
 0002:00000578       $SG47549                   000000014000a578     AccessInfo.obj
 0002:0000057c       $SG47562                   000000014000a57c     AccessInfo.obj
 0002:00000580       $SG47704                   000000014000a580     AccessInfo.obj
 0002:000005a8       $SG47705                   000000014000a5a8     AccessInfo.obj
 0002:000005c0       $SG47706                   000000014000a5c0     AccessInfo.obj
 0002:000005e8       $SG47707                   000000014000a5e8     AccessInfo.obj
 0002:00000618       $SG47708                   000000014000a618     AccessInfo.obj
 0002:00000648       $SG47709                   000000014000a648     AccessInfo.obj
 0002:00000678       $SG47713                   000000014000a678     AccessInfo.obj
 0002:000006a8       $SG47714                   000000014000a6a8     AccessInfo.obj
 0002:000006d0       $SG47717                   000000014000a6d0     AccessInfo.obj
 0002:000006ec       $SG47718                   000000014000a6ec     AccessInfo.obj
 0002:000006f0       $SG47719                   000000014000a6f0     AccessInfo.obj
 0002:00000708       $SG47722                   000000014000a708     AccessInfo.obj
 0002:00000730       $SG47723                   000000014000a730     AccessInfo.obj
 0002:00000750       $SG47724                   000000014000a750     AccessInfo.obj
 0002:00000768       $SG47725                   000000014000a768     AccessInfo.obj
 0002:00000780       $SG47726                   000000014000a780     AccessInfo.obj
 0002:000007a8       $SG47727                   000000014000a7a8     AccessInfo.obj
 0002:000007c0       $SG47728                   000000014000a7c0     AccessInfo.obj
 0002:000007e8       $SG47729                   000000014000a7e8     AccessInfo.obj
 0002:00000808       $SG47730                   000000014000a808     AccessInfo.obj
 0002:00000828       $SG47731                   000000014000a828     AccessInfo.obj
 0002:00000858       $SG47734                   000000014000a858     AccessInfo.obj
 0002:00000880       $SG47737                   000000014000a880     AccessInfo.obj
 0002:000008c0       $SG47740                   000000014000a8c0     AccessInfo.obj
 0002:000008e8       $SG47741                   000000014000a8e8     AccessInfo.obj
 0002:00000910       $SG47742                   000000014000a910     AccessInfo.obj
 0002:00000938       $SG47745                   000000014000a938     AccessInfo.obj
 0002:00000948       $SG47748                   000000014000a948     AccessInfo.obj
 0002:00000980       $SG47749                   000000014000a980     AccessInfo.obj
 0002:00000998       $SG47752                   000000014000a998     AccessInfo.obj
 0002:000009c0       $SG47753                   000000014000a9c0     AccessInfo.obj
 0002:000009e0       $SG47754                   000000014000a9e0     AccessInfo.obj
 0002:000009f8       $SG47757                   000000014000a9f8     AccessInfo.obj
 0002:00000a20       $SG47758                   000000014000aa20     AccessInfo.obj
 0002:00000a48       $SG47762                   000000014000aa48     AccessInfo.obj
 0002:00000a70       $SG47766                   000000014000aa70     AccessInfo.obj
 0002:00000a98       $SG47767                   000000014000aa98     AccessInfo.obj
 0002:00000ab8       $SG47768                   000000014000aab8     AccessInfo.obj
 0002:00000ad8       $SG47770                   000000014000aad8     AccessInfo.obj
 0002:00000b00       $SG47772                   000000014000ab00     AccessInfo.obj
 0002:00000b20       $SG47775                   000000014000ab20     AccessInfo.obj
 0002:00000b68       $SG47778                   000000014000ab68     AccessInfo.obj
 0002:00000ba8       $SG47781                   000000014000aba8     AccessInfo.obj
 0002:00000bd0       $SG47782                   000000014000abd0     AccessInfo.obj
 0002:00000bf0       $SG47783                   000000014000abf0     AccessInfo.obj
 0002:00000c10       $SG47784                   000000014000ac10     AccessInfo.obj
 0002:00000c40       $SG47786                   000000014000ac40     AccessInfo.obj
 0002:00000c60       $SG47787                   000000014000ac60     AccessInfo.obj
 0002:00000c88       $SG47788                   000000014000ac88     AccessInfo.obj
 0002:00000cb0       $SG47789                   000000014000acb0     AccessInfo.obj
 0002:00000cd8       $SG47791                   000000014000acd8     AccessInfo.obj
 0002:00000cf8       $SG47792                   000000014000acf8     AccessInfo.obj
 0002:00000d18       $SG47793                   000000014000ad18     AccessInfo.obj
 0002:00000d38       $SG47794                   000000014000ad38     AccessInfo.obj
 0002:00000d58       $SG47795                   000000014000ad58     AccessInfo.obj
 0002:00000d70       $SG47797                   000000014000ad70     AccessInfo.obj
 0002:00000d90       $SG47798                   000000014000ad90     AccessInfo.obj
 0002:00000db0       $SG47799                   000000014000adb0     AccessInfo.obj
 0002:00000dd0       $SG47802                   000000014000add0     AccessInfo.obj
 0002:00000df8       $SG47804                   000000014000adf8     AccessInfo.obj
 0002:00000e20       $SG47805                   000000014000ae20     AccessInfo.obj
 0002:00000e40       $SG47806                   000000014000ae40     AccessInfo.obj
 0002:00000e60       $SG47807                   000000014000ae60     AccessInfo.obj
 0002:00000e88       $SG47810                   000000014000ae88     AccessInfo.obj
 0002:00000eb8       $SG47813                   000000014000aeb8     AccessInfo.obj
 0002:00000ee0       $SG47814                   000000014000aee0     AccessInfo.obj
 0002:00000f00       $SG47815                   000000014000af00     AccessInfo.obj
 0002:00000f20       $SG47817                   000000014000af20     AccessInfo.obj
 0002:00000f48       $SG47819                   000000014000af48     AccessInfo.obj
 0002:00000f68       $SG47821                   000000014000af68     AccessInfo.obj
 0002:00000f88       $SG47823                   000000014000af88     AccessInfo.obj
 0002:00000fa8       $SG47827                   000000014000afa8     AccessInfo.obj
 0002:00000fd0       $SG47828                   000000014000afd0     AccessInfo.obj
 0002:00000ff0       $SG47829                   000000014000aff0     AccessInfo.obj
 0002:00001018       $SG47830                   000000014000b018     AccessInfo.obj
 0002:00001040       $SG47831                   000000014000b040     AccessInfo.obj
 0002:00001068       $SG47832                   000000014000b068     AccessInfo.obj
 0002:00001088       $SG47833                   000000014000b088     AccessInfo.obj
 0002:000010a8       $SG47836                   000000014000b0a8     AccessInfo.obj
 0002:000010d8       $SG47837                   000000014000b0d8     AccessInfo.obj
 0002:00001108       $SG47838                   000000014000b108     AccessInfo.obj
 0002:00001120       $SG47839                   000000014000b120     AccessInfo.obj
 0002:00001138       $SG47840                   000000014000b138     AccessInfo.obj
 0002:00001158       $SG47841                   000000014000b158     AccessInfo.obj
 0002:00001170       $SG47844                   000000014000b170     AccessInfo.obj
 0002:000011b8       $SG47847                   000000014000b1b8     AccessInfo.obj
 0002:000011e0       $SG47848                   000000014000b1e0     AccessInfo.obj
 0002:000011f8       $SG47849                   000000014000b1f8     AccessInfo.obj
 0002:00001210       $SG47852                   000000014000b210     AccessInfo.obj
 0002:00001240       $SG47853                   000000014000b240     AccessInfo.obj
 0002:00001268       $SG47854                   000000014000b268     AccessInfo.obj
 0002:00001290       $SG47855                   000000014000b290     AccessInfo.obj
 0002:000012b8       $SG47856                   000000014000b2b8     AccessInfo.obj
 0002:000012d8       $SG47859                   000000014000b2d8     AccessInfo.obj
 0002:00001310       $SG47860                   000000014000b310     AccessInfo.obj
 0002:00001328       $SG47861                   000000014000b328     AccessInfo.obj
 0002:00001330       $SG47864                   000000014000b330     AccessInfo.obj
 0002:00001360       $SG47865                   000000014000b360     AccessInfo.obj
 0002:00001388       $SG47866                   000000014000b388     AccessInfo.obj
 0002:000013a0       $SG47867                   000000014000b3a0     AccessInfo.obj
 0002:000013b8       $SG47868                   000000014000b3b8     AccessInfo.obj
 0002:000013d8       $SG47869                   000000014000b3d8     AccessInfo.obj
 0002:000013f0       $SG47872                   000000014000b3f0     AccessInfo.obj
 0002:00001420       $SG47875                   000000014000b420     AccessInfo.obj
 0002:00001448       $SG47876                   000000014000b448     AccessInfo.obj
 0002:00001460       $SG47877                   000000014000b460     AccessInfo.obj
 0002:00001478       $SG47879                   000000014000b478     AccessInfo.obj
 0002:000014a0       $SG47881                   000000014000b4a0     AccessInfo.obj
 0002:000014c8       $SG47882                   000000014000b4c8     AccessInfo.obj
 0002:000014e8       $SG47883                   000000014000b4e8     AccessInfo.obj
 0002:00001500       $SG47885                   000000014000b500     AccessInfo.obj
 0002:00001528       $SG47886                   000000014000b528     AccessInfo.obj
 0002:00001548       $SG47887                   000000014000b548     AccessInfo.obj
 0002:00001568       $SG47888                   000000014000b568     AccessInfo.obj
 0002:00001590       $SG47890                   000000014000b590     AccessInfo.obj
 0002:000015d0       $SG47893                   000000014000b5d0     AccessInfo.obj
 0002:000015f0       $SG47895                   000000014000b5f0     AccessInfo.obj
 0002:00001610       $SG47896                   000000014000b610     AccessInfo.obj
 0002:00001628       $SG47897                   000000014000b628     AccessInfo.obj
 0002:00001644       $SG47899                   000000014000b644     AccessInfo.obj
 0002:00001650       $SG47900                   000000014000b650     AccessInfo.obj
 0002:00001660       $SG47901                   000000014000b660     AccessInfo.obj
 0002:00001680       $SG47902                   000000014000b680     AccessInfo.obj
 0002:00001688       $SG47903                   000000014000b688     AccessInfo.obj
 0002:00001694       $SG47904                   000000014000b694     AccessInfo.obj
 0002:000016a0       $SG47905                   000000014000b6a0     AccessInfo.obj
 0002:000016b0       $SG47906                   000000014000b6b0     AccessInfo.obj
 0002:000016c0       $SG47907                   000000014000b6c0     AccessInfo.obj
 0002:000016c8       $SG47908                   000000014000b6c8     AccessInfo.obj
 0002:000016d8       $SG47909                   000000014000b6d8     AccessInfo.obj
 0002:000016ec       $SG47910                   000000014000b6ec     AccessInfo.obj
 0002:000016f8       $SG47911                   000000014000b6f8     AccessInfo.obj
 0002:00001708       $SG47912                   000000014000b708     AccessInfo.obj
 0002:00001718       $SG47913                   000000014000b718     AccessInfo.obj
 0002:00001720       $SG47914                   000000014000b720     AccessInfo.obj
 0002:00001730       $SG47915                   000000014000b730     AccessInfo.obj
 0002:00001740       $SG47916                   000000014000b740     AccessInfo.obj
 0002:00001748       $SG47917                   000000014000b748     AccessInfo.obj
 0002:00001770       $SG47918                   000000014000b770     AccessInfo.obj
 0002:00001798       $SG47919                   000000014000b798     AccessInfo.obj
 0002:000017b8       $SG47920                   000000014000b7b8     AccessInfo.obj
 0002:000017d8       $SG47921                   000000014000b7d8     AccessInfo.obj
 0002:00001800       $SG47922                   000000014000b800     AccessInfo.obj
 0002:00001820       $SG47923                   000000014000b820     AccessInfo.obj
 0002:00001840       $SG47924                   000000014000b840     AccessInfo.obj
 0002:00001860       $SG47925                   000000014000b860     AccessInfo.obj
 0002:00001880       $SG47926                   000000014000b880     AccessInfo.obj
 0002:000018a0       $SG47927                   000000014000b8a0     AccessInfo.obj
 0002:000018c8       $SG47930                   000000014000b8c8     AccessInfo.obj
 0002:000018e8       $SG47931                   000000014000b8e8     AccessInfo.obj
 0002:00001918       $SG47932                   000000014000b918     AccessInfo.obj
 0002:00001938       $SG47934                   000000014000b938     AccessInfo.obj
 0002:00001970       $SG47936                   000000014000b970     AccessInfo.obj
 0002:000019b0       $SG47939                   000000014000b9b0     AccessInfo.obj
 0002:000019d0       $SG47941                   000000014000b9d0     AccessInfo.obj
 0002:000019f0       $SG47942                   000000014000b9f0     AccessInfo.obj
 0002:00001a08       $SG47943                   000000014000ba08     AccessInfo.obj
 0002:00001a24       $SG47945                   000000014000ba24     AccessInfo.obj
 0002:00001a30       $SG47946                   000000014000ba30     AccessInfo.obj
 0002:00001a40       $SG47947                   000000014000ba40     AccessInfo.obj
 0002:00001a60       $SG47948                   000000014000ba60     AccessInfo.obj
 0002:00001a68       $SG47949                   000000014000ba68     AccessInfo.obj
 0002:00001a74       $SG47950                   000000014000ba74     AccessInfo.obj
 0002:00001a80       $SG47951                   000000014000ba80     AccessInfo.obj
 0002:00001a90       $SG47952                   000000014000ba90     AccessInfo.obj
 0002:00001aa0       $SG47953                   000000014000baa0     AccessInfo.obj
 0002:00001aa8       $SG47954                   000000014000baa8     AccessInfo.obj
 0002:00001ab8       $SG47955                   000000014000bab8     AccessInfo.obj
 0002:00001acc       $SG47956                   000000014000bacc     AccessInfo.obj
 0002:00001ad8       $SG47957                   000000014000bad8     AccessInfo.obj
 0002:00001ae8       $SG47958                   000000014000bae8     AccessInfo.obj
 0002:00001af8       $SG47959                   000000014000baf8     AccessInfo.obj
 0002:00001b00       $SG47960                   000000014000bb00     AccessInfo.obj
 0002:00001b10       $SG47961                   000000014000bb10     AccessInfo.obj
 0002:00001b20       $SG47962                   000000014000bb20     AccessInfo.obj
 0002:00001b28       $SG47963                   000000014000bb28     AccessInfo.obj
 0002:00001b50       $SG47964                   000000014000bb50     AccessInfo.obj
 0002:00001b78       $SG47965                   000000014000bb78     AccessInfo.obj
 0002:00001b98       $SG47966                   000000014000bb98     AccessInfo.obj
 0002:00001bb8       $SG47967                   000000014000bbb8     AccessInfo.obj
 0002:00001be0       $SG47968                   000000014000bbe0     AccessInfo.obj
 0002:00001c00       $SG47969                   000000014000bc00     AccessInfo.obj
 0002:00001c20       $SG47970                   000000014000bc20     AccessInfo.obj
 0002:00001c40       $SG47971                   000000014000bc40     AccessInfo.obj
 0002:00001c60       $SG47972                   000000014000bc60     AccessInfo.obj
 0002:00001c80       $SG47973                   000000014000bc80     AccessInfo.obj
 0002:00001ca8       $SG47976                   000000014000bca8     AccessInfo.obj
 0002:00001cc8       $SG47977                   000000014000bcc8     AccessInfo.obj
 0002:00001d00       $SG55324                   000000014000bd00     jaccesswalker.obj
 0002:00001d02       $SG55372                   000000014000bd02     jaccesswalker.obj
 0002:00001d03       $SG55446                   000000014000bd03     jaccesswalker.obj
 0002:00001d04       $SG55549                   000000014000bd04     jaccesswalker.obj
 0002:00001d08       $SG55325                   000000014000bd08     jaccesswalker.obj
 0002:00001d20       $SG55326                   000000014000bd20     jaccesswalker.obj
 0002:00001d40       $SG55412                   000000014000bd40     jaccesswalker.obj
 0002:00001d4c       $SG55447                   000000014000bd4c     jaccesswalker.obj
 0002:00001d58       $SG55475                   000000014000bd58     jaccesswalker.obj
 0002:00001d60       $SG55476                   000000014000bd60     jaccesswalker.obj
 0002:00001d78       $SG55499                   000000014000bd78     jaccesswalker.obj
 0002:00001d88       $SG55506                   000000014000bd88     jaccesswalker.obj
 0002:00001d98       $SG55510                   000000014000bd98     jaccesswalker.obj
 0002:00001da8       $SG55512                   000000014000bda8     jaccesswalker.obj
 0002:00001db8       $SG55515                   000000014000bdb8     jaccesswalker.obj
 0002:00001dc8       $SG55517                   000000014000bdc8     jaccesswalker.obj
 0002:00001dd8       $SG55519                   000000014000bdd8     jaccesswalker.obj
 0002:00001de8       $SG55524                   000000014000bde8     jaccesswalker.obj
 0002:00001df8       $SG55526                   000000014000bdf8     jaccesswalker.obj
 0002:00001e08       $SG55529                   000000014000be08     jaccesswalker.obj
 0002:00001e18       $SG55550                   000000014000be18     jaccesswalker.obj
 0002:00001e28       $SG55597                   000000014000be28     jaccesswalker.obj
 0002:00001e2c       $SG55598                   000000014000be2c     jaccesswalker.obj
 0002:00001e30       $SG55599                   000000014000be30     jaccesswalker.obj
 0002:00001e40       $SG55600                   000000014000be40     jaccesswalker.obj
 0002:00001e88       $SG55630                   000000014000be88     jaccesswalker.obj
 0002:00001ea8       $SG55632                   000000014000bea8     jaccesswalker.obj
 0002:00001ec8       GS_ExceptionPointers       000000014000bec8     MSVCRT:gs_report.obj
 0002:00002788       $unwind$initializeAccessBridge 000000014000c788     AccessBridgeCalls.obj
 0002:00002790       $unwind$shutdownAccessBridge 000000014000c790     AccessBridgeCalls.obj
 0002:00002798       $unwind$IsJavaWindow       000000014000c798     AccessBridgeCalls.obj
 0002:000027a0       $unwind$GetAccessibleContextFromHWND 000000014000c7a0     AccessBridgeCalls.obj
 0002:000027a8       $unwind$getHWNDFromAccessibleContext 000000014000c7a8     AccessBridgeCalls.obj
 0002:000027b0       $unwind$SetJavaShutdown    000000014000c7b0     AccessBridgeCalls.obj
 0002:000027b8       $unwind$SetFocusGained     000000014000c7b8     AccessBridgeCalls.obj
 0002:000027c0       $unwind$SetFocusLost       000000014000c7c0     AccessBridgeCalls.obj
 0002:000027c8       $unwind$SetCaretUpdate     000000014000c7c8     AccessBridgeCalls.obj
 0002:000027d0       $unwind$SetMouseClicked    000000014000c7d0     AccessBridgeCalls.obj
 0002:000027d8       $unwind$SetMouseEntered    000000014000c7d8     AccessBridgeCalls.obj
 0002:000027e0       $unwind$SetMouseExited     000000014000c7e0     AccessBridgeCalls.obj
 0002:000027e8       $unwind$SetMousePressed    000000014000c7e8     AccessBridgeCalls.obj
 0002:000027f0       $unwind$SetMouseReleased   000000014000c7f0     AccessBridgeCalls.obj
 0002:000027f8       $unwind$SetMenuCanceled    000000014000c7f8     AccessBridgeCalls.obj
 0002:00002800       $unwind$SetMenuDeselected  000000014000c800     AccessBridgeCalls.obj
 0002:00002808       $unwind$SetMenuSelected    000000014000c808     AccessBridgeCalls.obj
 0002:00002810       $unwind$SetPopupMenuCanceled 000000014000c810     AccessBridgeCalls.obj
 0002:00002818       $unwind$SetPopupMenuWillBecomeInvisible 000000014000c818     AccessBridgeCalls.obj
 0002:00002820       $unwind$SetPopupMenuWillBecomeVisible 000000014000c820     AccessBridgeCalls.obj
 0002:00002828       $unwind$SetPropertyNameChange 000000014000c828     AccessBridgeCalls.obj
 0002:00002830       $unwind$SetPropertyDescriptionChange 000000014000c830     AccessBridgeCalls.obj
 0002:00002838       $unwind$SetPropertyStateChange 000000014000c838     AccessBridgeCalls.obj
 0002:00002840       $unwind$SetPropertyValueChange 000000014000c840     AccessBridgeCalls.obj
 0002:00002848       $unwind$SetPropertySelectionChange 000000014000c848     AccessBridgeCalls.obj
 0002:00002850       $unwind$SetPropertyTextChange 000000014000c850     AccessBridgeCalls.obj
 0002:00002858       $unwind$SetPropertyCaretChange 000000014000c858     AccessBridgeCalls.obj
 0002:00002860       $unwind$SetPropertyVisibleDataChange 000000014000c860     AccessBridgeCalls.obj
 0002:00002868       $unwind$SetPropertyChildChange 000000014000c868     AccessBridgeCalls.obj
 0002:00002870       $unwind$SetPropertyActiveDescendentChange 000000014000c870     AccessBridgeCalls.obj
 0002:00002878       $unwind$SetPropertyTableModelChange 000000014000c878     AccessBridgeCalls.obj
 0002:00002880       $unwind$ReleaseJavaObject  000000014000c880     AccessBridgeCalls.obj
 0002:00002888       $unwind$GetVersionInfo     000000014000c888     AccessBridgeCalls.obj
 0002:00002890       $unwind$GetAccessibleContextAt 000000014000c890     AccessBridgeCalls.obj
 0002:00002898       $unwind$GetAccessibleContextWithFocus 000000014000c898     AccessBridgeCalls.obj
 0002:000028a0       $unwind$GetAccessibleContextInfo 000000014000c8a0     AccessBridgeCalls.obj
 0002:000028a8       $unwind$GetAccessibleChildFromContext 000000014000c8a8     AccessBridgeCalls.obj
 0002:000028b0       $unwind$GetAccessibleParentFromContext 000000014000c8b0     AccessBridgeCalls.obj
 0002:000028b8       $unwind$GetAccessibleTextInfo 000000014000c8b8     AccessBridgeCalls.obj
 0002:000028c0       $unwind$GetAccessibleTextItems 000000014000c8c0     AccessBridgeCalls.obj
 0002:000028c8       $unwind$GetAccessibleTextSelectionInfo 000000014000c8c8     AccessBridgeCalls.obj
 0002:000028d0       $unwind$GetAccessibleTextAttributes 000000014000c8d0     AccessBridgeCalls.obj
 0002:000028d8       $unwind$GetAccessibleTextRect 000000014000c8d8     AccessBridgeCalls.obj
 0002:000028e0       $unwind$GetAccessibleTextLineBounds 000000014000c8e0     AccessBridgeCalls.obj
 0002:000028e8       $unwind$GetAccessibleTextRange 000000014000c8e8     AccessBridgeCalls.obj
 0002:000028f0       $unwind$getAccessibleTableInfo 000000014000c8f0     AccessBridgeCalls.obj
 0002:000028f8       $unwind$getAccessibleTableCellInfo 000000014000c8f8     AccessBridgeCalls.obj
 0002:00002900       $unwind$getAccessibleTableRowHeader 000000014000c900     AccessBridgeCalls.obj
 0002:00002908       $unwind$getAccessibleTableColumnHeader 000000014000c908     AccessBridgeCalls.obj
 0002:00002910       $unwind$getAccessibleTableRowDescription 000000014000c910     AccessBridgeCalls.obj
 0002:00002918       $unwind$getAccessibleTableColumnDescription 000000014000c918     AccessBridgeCalls.obj
 0002:00002920       $unwind$getAccessibleTableRowSelectionCount 000000014000c920     AccessBridgeCalls.obj
 0002:00002928       $unwind$isAccessibleTableRowSelected 000000014000c928     AccessBridgeCalls.obj
 0002:00002930       $unwind$getAccessibleTableRowSelections 000000014000c930     AccessBridgeCalls.obj
 0002:00002938       $unwind$getAccessibleTableColumnSelectionCount 000000014000c938     AccessBridgeCalls.obj
 0002:00002940       $unwind$isAccessibleTableColumnSelected 000000014000c940     AccessBridgeCalls.obj
 0002:00002948       $unwind$getAccessibleTableColumnSelections 000000014000c948     AccessBridgeCalls.obj
 0002:00002950       $unwind$getAccessibleTableRow 000000014000c950     AccessBridgeCalls.obj
 0002:00002958       $unwind$getAccessibleTableColumn 000000014000c958     AccessBridgeCalls.obj
 0002:00002960       $unwind$getAccessibleTableIndex 000000014000c960     AccessBridgeCalls.obj
 0002:00002968       $unwind$getAccessibleRelationSet 000000014000c968     AccessBridgeCalls.obj
 0002:00002970       $unwind$getAccessibleHypertext 000000014000c970     AccessBridgeCalls.obj
 0002:00002978       $unwind$activateAccessibleHyperlink 000000014000c978     AccessBridgeCalls.obj
 0002:00002980       $unwind$getAccessibleHyperlinkCount 000000014000c980     AccessBridgeCalls.obj
 0002:00002988       $unwind$getAccessibleHypertextExt 000000014000c988     AccessBridgeCalls.obj
 0002:00002990       $unwind$getAccessibleHypertextLinkIndex 000000014000c990     AccessBridgeCalls.obj
 0002:00002998       $unwind$getAccessibleHyperlink 000000014000c998     AccessBridgeCalls.obj
 0002:000029a0       $unwind$getAccessibleKeyBindings 000000014000c9a0     AccessBridgeCalls.obj
 0002:000029a8       $unwind$getAccessibleIcons 000000014000c9a8     AccessBridgeCalls.obj
 0002:000029b0       $unwind$getAccessibleActions 000000014000c9b0     AccessBridgeCalls.obj
 0002:000029b8       $unwind$doAccessibleActions 000000014000c9b8     AccessBridgeCalls.obj
 0002:000029c0       $unwind$IsSameObject       000000014000c9c0     AccessBridgeCalls.obj
 0002:000029c8       $unwind$setTextContents    000000014000c9c8     AccessBridgeCalls.obj
 0002:000029d0       $unwind$getParentWithRole  000000014000c9d0     AccessBridgeCalls.obj
 0002:000029d8       $unwind$getParentWithRoleElseRoot 000000014000c9d8     AccessBridgeCalls.obj
 0002:000029e0       $unwind$getTopLevelObject  000000014000c9e0     AccessBridgeCalls.obj
 0002:000029e8       $unwind$getObjectDepth     000000014000c9e8     AccessBridgeCalls.obj
 0002:000029f0       $unwind$getActiveDescendent 000000014000c9f0     AccessBridgeCalls.obj
 0002:000029f8       $unwind$GetCurrentAccessibleValueFromContext 000000014000c9f8     AccessBridgeCalls.obj
 0002:00002a00       $unwind$GetMaximumAccessibleValueFromContext 000000014000ca00     AccessBridgeCalls.obj
 0002:00002a08       $unwind$GetMinimumAccessibleValueFromContext 000000014000ca08     AccessBridgeCalls.obj
 0002:00002a10       $unwind$GetAccessibleSelectionFromContext 000000014000ca10     AccessBridgeCalls.obj
 0002:00002a18       $unwind$GetAccessibleSelectionCountFromContext 000000014000ca18     AccessBridgeCalls.obj
 0002:00002a20       $unwind$IsAccessibleChildSelectedFromContext 000000014000ca20     AccessBridgeCalls.obj
 0002:00002a28       $unwind$RemoveAccessibleSelectionFromContext 000000014000ca28     AccessBridgeCalls.obj
 0002:00002a30       $unwind$SelectAllAccessibleSelectionFromContext 000000014000ca30     AccessBridgeCalls.obj
 0002:00002a38       $unwind$getVirtualAccessibleName 000000014000ca38     AccessBridgeCalls.obj
 0002:00002a40       $unwind$requestFocus       000000014000ca40     AccessBridgeCalls.obj
 0002:00002a48       $unwind$selectTextRange    000000014000ca48     AccessBridgeCalls.obj
 0002:00002a50       $unwind$getTextAttributesInRange 000000014000ca50     AccessBridgeCalls.obj
 0002:00002a58       $unwind$getVisibleChildrenCount 000000014000ca58     AccessBridgeCalls.obj
 0002:00002a60       $unwind$getVisibleChildren 000000014000ca60     AccessBridgeCalls.obj
 0002:00002a68       $unwind$setCaretPosition   000000014000ca68     AccessBridgeCalls.obj
 0002:00002a70       $unwind$getCaretLocation   000000014000ca70     AccessBridgeCalls.obj
 0002:00002a78       $unwind$getEventsWaiting   000000014000ca78     AccessBridgeCalls.obj
 0002:00002a80       $unwind$addAccessibleSelectionFromContext 000000014000ca80     AccessBridgeCalls.obj
 0002:00002a88       $unwind$clearAccessibleSelectionFromContext 000000014000ca88     AccessBridgeCalls.obj
 0002:00002a90       $unwind$printError         000000014000ca90     AccessBridgeDebug.obj
 0002:00002a98       $unwind$PrintDebugString   000000014000ca98     AccessBridgeDebug.obj
 0002:00002aa0       $unwind$wPrintJavaDebugString 000000014000caa0     AccessBridgeDebug.obj
 0002:00002aa8       $unwind$wPrintDebugString  000000014000caa8     AccessBridgeDebug.obj
 0002:00002ab0       $unwind$initializeFileLogger 000000014000cab0     AccessBridgeDebug.obj
 0002:00002ab8       $unwind$finalizeFileLogger 000000014000cab8     AccessBridgeDebug.obj
 0002:00002ac0       $unwind$getTimeStamp       000000014000cac0     AccessBridgeDebug.obj
 0002:00002ac8       $unwind$PrintJavaDebugString2 000000014000cac8     AccessBridgeDebug.obj
 0002:00002ad0       $unwind$_vfprintf_l        000000014000cad0     AccessBridgeDebug.obj
 0002:00002ad0       $unwind$_vfwprintf_l       000000014000cad0     AccessBridgeDebug.obj
 0002:00002ad0       $unwind$fprintf            000000014000cad0     AccessBridgeDebug.obj
 0002:00002ad0       $unwind$printf             000000014000cad0     AccessBridgeDebug.obj
 0002:00002ad0       $unwind$snprintf           000000014000cad0     AccessInfo.obj
 0002:00002ad8       $unwind$vfprintf           000000014000cad8     AccessBridgeDebug.obj
 0002:00002ad8       $unwind$vfwprintf          000000014000cad8     AccessBridgeDebug.obj
 0002:00002ae0       $unwind$?initBroadcastMessageIDs@@YAHXZ 000000014000cae0     AccessBridgeMessages.obj
 0002:00002ae8       $unwind$vsnprintf          000000014000cae8     AccessInfo.obj
 0002:00002af0       $unwind$?getTimeAndDate@@YAPEADXZ 000000014000caf0     AccessInfo.obj
 0002:00002afc       $unwind$?displayAndLog@@YAXPEAUHWND__@@HPEAU_iobuf@@PEADZZ 000000014000cafc     AccessInfo.obj
 0002:00002b0c       $unwind$?logString@@YAXPEAU_iobuf@@PEBDZZ 000000014000cb0c     AccessInfo.obj
 0002:00002b1c       $unwind$?getAccessibleInfo@@YAPEADJ_JPEADH@Z 000000014000cb1c     AccessInfo.obj
 0002:00002b24       $unwind$?getAccessibleInfo@@YAPEADJ_JHHPEADH@Z 000000014000cb24     AccessInfo.obj
 0002:00002b38       $unwind$localtime          000000014000cb38     AccessInfo.obj
 0002:00002b40       $unwind$time               000000014000cb40     AccessInfo.obj
 0002:00002b48       $unwind$?appendToBuffer@@YAHPEAD_KPEBDZZ 000000014000cb48     AccessInfo.obj
 0002:00002b58       $unwind$WinMain            000000014000cb58     jaccesswalker.obj
 0002:00002b60       $unwind$??1AccessibleNode@@QEAA@XZ 000000014000cb60     jaccesswalker.obj
 0002:00002b68       $unwind$?setAccessibleName@AccessibleNode@@QEAAXPEAD@Z 000000014000cb68     jaccesswalker.obj
 0002:00002b70       $unwind$?setAccessibleRole@AccessibleNode@@QEAAXPEAD@Z 000000014000cb70     jaccesswalker.obj
 0002:00002b78       $unwind$?displayAPIWindow@AccessibleNode@@QEAAHXZ 000000014000cb78     jaccesswalker.obj
 0002:00002b88       $unwind$??0Jaccesswalker@@QEAA@H@Z 000000014000cb88     jaccesswalker.obj
 0002:00002b90       $unwind$?buildAccessibilityTree@Jaccesswalker@@QEAAXXZ 000000014000cb90     jaccesswalker.obj
 0002:00002b98       $unwind$?addComponentNodes@Jaccesswalker@@QEAAXJ_JPEAVAccessibleNode@@PEAUHWND__@@PEAU_TREEITEM@@2@Z 000000014000cb98     jaccesswalker.obj
 0002:00002bb0       $cppxdata$?addComponentNodes@Jaccesswalker@@QEAAXJ_JPEAVAccessibleNode@@PEAUHWND__@@PEAU_TREEITEM@@2@Z 000000014000cbb0     jaccesswalker.obj
 0002:00002bb9       $stateUnwindMap$?addComponentNodes@Jaccesswalker@@QEAAXJ_JPEAVAccessibleNode@@PEAUHWND__@@PEAU_TREEITEM@@2@Z 000000014000cbb9     jaccesswalker.obj
 0002:00002bbf       $ip2state$?addComponentNodes@Jaccesswalker@@QEAAXJ_JPEAVAccessibleNode@@PEAUHWND__@@PEAU_TREEITEM@@2@Z 000000014000cbbf     jaccesswalker.obj
 0002:00002bc8       $unwind$?dtor$0@?0??addComponentNodes@Jaccesswalker@@QEAAXJ_JPEAVAccessibleNode@@PEAUHWND__@@PEAU_TREEITEM@@2@Z@4HA 000000014000cbc8     jaccesswalker.obj
 0002:00002bd0       $unwind$?WinProc@@YA_JPEAUHWND__@@I_K_J@Z 000000014000cbd0     jaccesswalker.obj
 0002:00002bd8       $unwind$?EnumWndProc@@YAHPEAUHWND__@@_J@Z 000000014000cbd8     jaccesswalker.obj
 0002:00002bec       $unwind$?EnumChildProc@@YAHPEAUHWND__@@_J@Z 000000014000cbec     jaccesswalker.obj
 0002:00002bf4       $unwind$?CreateATreeView@@YAPEAUHWND__@@PEAU1@@Z 000000014000cbf4     jaccesswalker.obj
 0002:00002c04       $unwind$?AccessInfoWindowProc@@YA_JPEAUHWND__@@IIJ@Z 000000014000cc04     jaccesswalker.obj
 0002:00002c14       $unwind$?IsInaccessibleJavaWindow@@YAHQEAUHWND__@@@Z 000000014000cc14     jaccesswalker.obj
 0002:00002c28       $unwind$__report_securityfailure 000000014000cc28     MSVCRT:gs_report.obj
 0002:00002c30       $unwind$__scrt_initialize_default_local_stdio_options 000000014000cc30     MSVCRT:default_local_stdio_options.obj
 0002:00002c30       $unwind$?post_pgo_initialization@@YAHXZ 000000014000cc30     MSVCRT:exe_winmain.obj
 0002:00002c30       $unwind$?pre_cpp_initialization@@YAXXZ 000000014000cc30     MSVCRT:exe_winmain.obj
 0002:00002c30       $unwind$WinMainCRTStartup  000000014000cc30     MSVCRT:exe_winmain.obj
 0002:00002c30       $unwind$__report_rangecheckfailure 000000014000cc30     MSVCRT:gs_report.obj
 0002:00002c30       $unwind$__GSHandlerCheck   000000014000cc30     MSVCRT:gshandler.obj
 0002:00002c30       $unwind$__scrt_acquire_startup_lock 000000014000cc30     MSVCRT:utility.obj
 0002:00002c30       $unwind$__scrt_initialize_crt 000000014000cc30     MSVCRT:utility.obj
 0002:00002c30       $unwind$atexit             000000014000cc30     MSVCRT:utility.obj
 0002:00002c30       $unwind$__scrt_is_managed_app 000000014000cc30     MSVCRT:utility_desktop.obj
 0002:00002c38       $unwind$__report_gsfailure 000000014000cc38     MSVCRT:gs_report.obj
 0002:00002c40       $unwind$capture_current_context 000000014000cc40     MSVCRT:gs_report.obj
 0002:00002c4c       $unwind$capture_previous_context 000000014000cc4c     MSVCRT:gs_report.obj
 0002:00002c58       $unwind$?pre_c_initialization@@YAHXZ 000000014000cc58     MSVCRT:exe_winmain.obj
 0002:00002c58       $unwind$__raise_securityfailure 000000014000cc58     MSVCRT:gs_report.obj
 0002:00002c58       $unwind$??2@YAPEAX_K@Z     000000014000cc58     MSVCRT:new_scalar.obj
 0002:00002c58       $unwind$??_Gtype_info@@UEAAPEAXI@Z 000000014000cc58     MSVCRT:std_type_info_static.obj
 0002:00002c58       $unwind$??0bad_alloc@std@@QEAA@AEBV01@@Z 000000014000cc58     MSVCRT:throw_bad_alloc.obj
 0002:00002c58       $unwind$??0bad_array_new_length@std@@QEAA@AEBV01@@Z 000000014000cc58     MSVCRT:throw_bad_alloc.obj
 0002:00002c58       $unwind$??0exception@std@@QEAA@AEBV01@@Z 000000014000cc58     MSVCRT:throw_bad_alloc.obj
 0002:00002c58       $unwind$__scrt_initialize_onexit_tables 000000014000cc58     MSVCRT:utility.obj
 0002:00002c58       $unwind$__scrt_release_startup_lock 000000014000cc58     MSVCRT:utility.obj
 0002:00002c58       $unwind$__scrt_uninitialize_crt 000000014000cc58     MSVCRT:utility.obj
 0002:00002c58       $unwind$_onexit            000000014000cc58     MSVCRT:utility.obj
 0002:00002c60       $unwind$__GSHandlerCheckCommon 000000014000cc60     MSVCRT:gshandler.obj
 0002:00002c68       $xdatasym                  000000014000cc68     MSVCRT:chkstk.obj
 0002:00002c70       $xdatasym                  000000014000cc70     MSVCRT:amdsecgs.obj
 0002:00002c74       $unwind$__GSHandlerCheck_EH4 000000014000cc74     MSVCRT:gshandlereh4.obj
 0002:00002c8c       $unwind$?__scrt_common_main_seh@@YAHXZ 000000014000cc8c     MSVCRT:exe_winmain.obj
 0002:00002cc0       $unwind$?filt$0@?0??__scrt_common_main_seh@@YAHXZ@4HA 000000014000ccc0     MSVCRT:exe_winmain.obj
 0002:00002cc8       $unwind$_RTC_Initialize    000000014000ccc8     MSVCRT:initsect.obj
 0002:00002cc8       $unwind$_RTC_Terminate     000000014000ccc8     MSVCRT:initsect.obj
 0002:00002cc8       $unwind$??_Gbad_alloc@std@@UEAAPEAXI@Z 000000014000ccc8     MSVCRT:throw_bad_alloc.obj
 0002:00002cc8       $unwind$??_Gbad_array_new_length@std@@UEAAPEAXI@Z 000000014000ccc8     MSVCRT:throw_bad_alloc.obj
 0002:00002cc8       $unwind$??_Gexception@std@@UEAAPEAXI@Z 000000014000ccc8     MSVCRT:throw_bad_alloc.obj
 0002:00002cc8       $unwind$__scrt_unhandled_exception_filter 000000014000ccc8     MSVCRT:utility_desktop.obj
 0002:00002cd4       $unwind$?__scrt_throw_std_bad_alloc@@YAXXZ 000000014000ccd4     MSVCRT:throw_bad_alloc.obj
 0002:00002cd4       $unwind$?__scrt_throw_std_bad_array_new_length@@YAXXZ 000000014000ccd4     MSVCRT:throw_bad_alloc.obj
 0002:00002cdc       $unwind$__scrt_is_nonwritable_in_current_image 000000014000ccdc     MSVCRT:utility.obj
 0002:00002cfc       $unwind$__scrt_is_nonwritable_in_current_image$filt$0 000000014000ccfc     MSVCRT:utility.obj
 0002:00002d04       $unwind$__security_init_cookie 000000014000cd04     MSVCRT:gs_support.obj
 0002:00002d10       $unwind$__scrt_get_show_window_mode 000000014000cd10     MSVCRT:utility_desktop.obj
 0002:00002d18       $unwind$__scrt_fastfail    000000014000cd18     MSVCRT:utility_desktop.obj
 0002:00002d28       $unwind$__isa_available_init 000000014000cd28     MSVCRT:cpu_disp.obj
 0002:00002d40       $xdatasym                  000000014000cd40     MSVCRT:guard_dispatch.obj
 0002:00002d48       $xdatasym                  000000014000cd48     MSVCRT:guard_xfg_dispatch.obj
 0002:00003320       .idata$6                   000000014000d320     comctl32:COMCTL32.dll
 0002:00003340       .idata$6                   000000014000d340     gdi32:GDI32.dll
 0002:00003514       .idata$6                   000000014000d514     user32:USER32.dll
 0002:000036ee       .idata$6                   000000014000d6ee     kernel32:KERNEL32.dll
 0002:000037ba       .idata$6                   000000014000d7ba     vcruntime:VCRUNTIME140.dll
 0002:000037cc       .idata$6                   000000014000d7cc     vcruntime:VCRUNTIME140_1.dll
 0002:00003a7e       .idata$6                   000000014000da7e     ucrt:api-ms-win-crt-string-l1-1-0.dll
 0002:00003aa0       .idata$6                   000000014000daa0     ucrt:api-ms-win-crt-stdio-l1-1-0.dll
 0002:00003ac0       .idata$6                   000000014000dac0     ucrt:api-ms-win-crt-environment-l1-1-0.dll
 0002:00003ae6       .idata$6                   000000014000dae6     ucrt:api-ms-win-crt-time-l1-1-0.dll
 0002:00003b06       .idata$6                   000000014000db06     ucrt:api-ms-win-crt-heap-l1-1-0.dll
 0002:00003b26       .idata$6                   000000014000db26     ucrt:api-ms-win-crt-runtime-l1-1-0.dll
 0002:00003b48       .idata$6                   000000014000db48     ucrt:api-ms-win-crt-math-l1-1-0.dll
 0002:00003b68       .idata$6                   000000014000db68     ucrt:api-ms-win-crt-locale-l1-1-0.dll
 0003:00000000       $SG37887                   000000014000e000     AccessBridgeCalls.obj
 0003:00000018       $SG37891                   000000014000e018     AccessBridgeCalls.obj
 0003:00000028       $SG37893                   000000014000e028     AccessBridgeCalls.obj
 0003:00000040       $SG37895                   000000014000e040     AccessBridgeCalls.obj
 0003:00000058       $SG37897                   000000014000e058     AccessBridgeCalls.obj
 0003:00000068       $SG37899                   000000014000e068     AccessBridgeCalls.obj
 0003:00000080       $SG37901                   000000014000e080     AccessBridgeCalls.obj
 0003:00000098       $SG37903                   000000014000e098     AccessBridgeCalls.obj
 0003:000000b0       $SG37905                   000000014000e0b0     AccessBridgeCalls.obj
 0003:000000c8       $SG37907                   000000014000e0c8     AccessBridgeCalls.obj
 0003:000000e0       $SG37909                   000000014000e0e0     AccessBridgeCalls.obj
 0003:000000f8       $SG37911                   000000014000e0f8     AccessBridgeCalls.obj
 0003:00000110       $SG37913                   000000014000e110     AccessBridgeCalls.obj
 0003:00000128       $SG37915                   000000014000e128     AccessBridgeCalls.obj
 0003:00000140       $SG37917                   000000014000e140     AccessBridgeCalls.obj
 0003:00000158       $SG37919                   000000014000e158     AccessBridgeCalls.obj
 0003:00000180       $SG37921                   000000014000e180     AccessBridgeCalls.obj
 0003:000001a0       $SG37923                   000000014000e1a0     AccessBridgeCalls.obj
 0003:000001b8       $SG37925                   000000014000e1b8     AccessBridgeCalls.obj
 0003:000001d8       $SG37927                   000000014000e1d8     AccessBridgeCalls.obj
 0003:000001f8       $SG37929                   000000014000e1f8     AccessBridgeCalls.obj
 0003:00000218       $SG37931                   000000014000e218     AccessBridgeCalls.obj
 0003:00000238       $SG37933                   000000014000e238     AccessBridgeCalls.obj
 0003:00000250       $SG37935                   000000014000e250     AccessBridgeCalls.obj
 0003:00000270       $SG37937                   000000014000e270     AccessBridgeCalls.obj
 0003:00000290       $SG37939                   000000014000e290     AccessBridgeCalls.obj
 0003:000002b0       $SG37941                   000000014000e2b0     AccessBridgeCalls.obj
 0003:000002d8       $SG37943                   000000014000e2d8     AccessBridgeCalls.obj
 0003:000002f8       $SG37945                   000000014000e2f8     AccessBridgeCalls.obj
 0003:00000310       $SG37947                   000000014000e310     AccessBridgeCalls.obj
 0003:00000320       $SG37949                   000000014000e320     AccessBridgeCalls.obj
 0003:00000330       $SG37951                   000000014000e330     AccessBridgeCalls.obj
 0003:00000340       $SG37953                   000000014000e340     AccessBridgeCalls.obj
 0003:00000360       $SG37955                   000000014000e360     AccessBridgeCalls.obj
 0003:00000380       $SG37957                   000000014000e380     AccessBridgeCalls.obj
 0003:00000398       $SG37959                   000000014000e398     AccessBridgeCalls.obj
 0003:000003b8       $SG37961                   000000014000e3b8     AccessBridgeCalls.obj
 0003:000003d8       $SG37963                   000000014000e3d8     AccessBridgeCalls.obj
 0003:000003f8       $SG37965                   000000014000e3f8     AccessBridgeCalls.obj
 0003:00000418       $SG37967                   000000014000e418     AccessBridgeCalls.obj
 0003:00000430       $SG37969                   000000014000e430     AccessBridgeCalls.obj
 0003:00000450       $SG37971                   000000014000e450     AccessBridgeCalls.obj
 0003:00000470       $SG37973                   000000014000e470     AccessBridgeCalls.obj
 0003:00000490       $SG37975                   000000014000e490     AccessBridgeCalls.obj
 0003:000004b8       $SG37977                   000000014000e4b8     AccessBridgeCalls.obj
 0003:000004e0       $SG37979                   000000014000e4e0     AccessBridgeCalls.obj
 0003:00000508       $SG37981                   000000014000e508     AccessBridgeCalls.obj
 0003:00000528       $SG37983                   000000014000e528     AccessBridgeCalls.obj
 0003:00000548       $SG37985                   000000014000e548     AccessBridgeCalls.obj
 0003:00000570       $SG37987                   000000014000e570     AccessBridgeCalls.obj
 0003:00000590       $SG37989                   000000014000e590     AccessBridgeCalls.obj
 0003:000005b8       $SG37991                   000000014000e5b8     AccessBridgeCalls.obj
 0003:000005d0       $SG37993                   000000014000e5d0     AccessBridgeCalls.obj
 0003:000005f0       $SG37995                   000000014000e5f0     AccessBridgeCalls.obj
 0003:00000608       $SG37997                   000000014000e608     AccessBridgeCalls.obj
 0003:00000628       $SG37999                   000000014000e628     AccessBridgeCalls.obj
 0003:00000640       $SG38001                   000000014000e640     AccessBridgeCalls.obj
 0003:00000660       $SG38003                   000000014000e660     AccessBridgeCalls.obj
 0003:00000680       $SG38005                   000000014000e680     AccessBridgeCalls.obj
 0003:000006a0       $SG38007                   000000014000e6a0     AccessBridgeCalls.obj
 0003:000006c0       $SG38009                   000000014000e6c0     AccessBridgeCalls.obj
 0003:000006d8       $SG38011                   000000014000e6d8     AccessBridgeCalls.obj
 0003:000006f8       $SG38013                   000000014000e6f8     AccessBridgeCalls.obj
 0003:00000710       $SG38015                   000000014000e710     AccessBridgeCalls.obj
 0003:00000728       $SG38017                   000000014000e728     AccessBridgeCalls.obj
 0003:00000740       $SG38019                   000000014000e740     AccessBridgeCalls.obj
 0003:00000758       $SG38021                   000000014000e758     AccessBridgeCalls.obj
 0003:00000770       $SG38023                   000000014000e770     AccessBridgeCalls.obj
 0003:00000790       $SG38025                   000000014000e790     AccessBridgeCalls.obj
 0003:000007b0       $SG38027                   000000014000e7b0     AccessBridgeCalls.obj
 0003:000007c8       $SG38029                   000000014000e7c8     AccessBridgeCalls.obj
 0003:000007e8       $SG38031                   000000014000e7e8     AccessBridgeCalls.obj
 0003:00000800       $SG38033                   000000014000e800     AccessBridgeCalls.obj
 0003:00000828       $SG38035                   000000014000e828     AccessBridgeCalls.obj
 0003:00000850       $SG38037                   000000014000e850     AccessBridgeCalls.obj
 0003:00000878       $SG38039                   000000014000e878     AccessBridgeCalls.obj
 0003:000008a0       $SG38041                   000000014000e8a0     AccessBridgeCalls.obj
 0003:000008c8       $SG38043                   000000014000e8c8     AccessBridgeCalls.obj
 0003:000008f0       $SG38045                   000000014000e8f0     AccessBridgeCalls.obj
 0003:00000918       $SG38047                   000000014000e918     AccessBridgeCalls.obj
 0003:00000940       $SG38049                   000000014000e940     AccessBridgeCalls.obj
 0003:00000968       $SG38051                   000000014000e968     AccessBridgeCalls.obj
 0003:00000990       $SG38053                   000000014000e990     AccessBridgeCalls.obj
 0003:000009a0       $SG38055                   000000014000e9a0     AccessBridgeCalls.obj
 0003:000009b8       $SG38057                   000000014000e9b8     AccessBridgeCalls.obj
 0003:000009d0       $SG38059                   000000014000e9d0     AccessBridgeCalls.obj
 0003:000009f0       $SG38061                   000000014000e9f0     AccessBridgeCalls.obj
 0003:00000a00       $SG38063                   000000014000ea00     AccessBridgeCalls.obj
 0003:00000a18       $SG38065                   000000014000ea18     AccessBridgeCalls.obj
 0003:00000a38       $SG38067                   000000014000ea38     AccessBridgeCalls.obj
 0003:00000a48       $SG38069                   000000014000ea48     AccessBridgeCalls.obj
 0003:00000a58       $SG38071                   000000014000ea58     AccessBridgeCalls.obj
 0003:00000a78       $SG38073                   000000014000ea78     AccessBridgeCalls.obj
 0003:00000a90       $SG38075                   000000014000ea90     AccessBridgeCalls.obj
 0003:00000aa8       $SG38077                   000000014000eaa8     AccessBridgeCalls.obj
 0003:00000ac0       $SG38079                   000000014000eac0     AccessBridgeCalls.obj
 0003:00000ad8       $SG38081                   000000014000ead8     AccessBridgeCalls.obj
 0003:00000af0       ?warning@?1??appendToBuffer@@YAHPEAD_KPEBDZZ@4PADA 000000014000eaf0     AccessInfo.obj
 0003:00000b60       ?szAppName@?1???0Jaccesswalker@@QEAA@H@Z@4PADA 000000014000eb60     jaccesswalker.obj
 0003:00000b70       ?szMenuName@?1???0Jaccesswalker@@QEAA@H@Z@4PADA 000000014000eb70     jaccesswalker.obj
 0003:00000d10       logFP                      000000014000ed10     AccessBridgeDebug.obj
 0003:00000d20       ?retbuf@?1??printError@@9@4PADA 000000014000ed20     AccessBridgeDebug.obj
 0003:00000e30       ?datebuf@?1??getTimeAndDate@@YAPEADXZ@4PADA 000000014000ee30     AccessInfo.obj
 0003:00000ed0       GS_ExceptionRecord         000000014000eed0     MSVCRT:gs_report.obj
 0003:00000f70       GS_ContextRecord           000000014000ef70     MSVCRT:gs_report.obj
 0003:00001450       ?is_initialized_as_dll@@3_NA 000000014000f450     MSVCRT:utility.obj
 0003:00001451       ?module_local_atexit_table_initialized@@3_NA 000000014000f451     MSVCRT:utility.obj
 0003:00001458       ?module_local_atexit_table@@3U_onexit_table_t@@A 000000014000f458     MSVCRT:utility.obj
 0003:00001470       ?module_local_at_quick_exit_table@@3U_onexit_table_t@@A 000000014000f470     MSVCRT:utility.obj
 0005:000001d0       $R000000                   00000001400111d0     jaccesswalker.exe.res
 0005:00000500       $R000330                   0000000140011500     jaccesswalker.exe.res
 0005:00000590       $R0003C0                   0000000140011590     jaccesswalker.exe.res
 0005:00000620       $R000450                   0000000140011620     jaccesswalker.exe.res
 0005:000006c0       $R0004F0                   00000001400116c0     jaccesswalker.exe.res
